:020000040000FA
:0408000064EF0BF0A6
:1008100003B273EF05F0F2B491EF05F09EB099EFDB
:1008200005F09EB2A1EF05F0F2A81AEF04F0F2B2C3
:1008300021EF04F0F2B01FEF04F013EF0BF0F2968B
:10084000F290CD90F2929EA02BEF04F00101533F65
:100850002BEF04F0542BB2C1B6F1B3C1B7F1B4C160
:10086000B8F1B5C1B9F1AEC1B2F1AFC1B3F1B0C128
:10087000B4F1B1C1B5F1AAC1AEF1ABC1AFF1ACC138
:10088000B0F1ADC1B1F1A6C1AAF1A7C1ABF1A8C148
:10089000ACF1A9C1ADF1A2C1A6F1A3C1A7F1A4C158
:1008A000A8F1A5C1A9F19EC1A2F19FC1A3F1A0C168
:1008B000A4F1A1C1A5F19AC19EF19BC19FF19CC178
:1008C000A0F19DC1A1F1CECF9AF1CFCF9BF153C141
:1008D0009CF154C19DF1CF6ACE6A0101536B546BF8
:1008E0009E90CD800FBC0F8E0FBA7AEF04F00F8A66
:1008F00013EF0BF013880F8C0FBEB7EF04F09AC103
:100900009EF19BC19FF19CC1A0F19DC1A1F19EC12F
:10091000A2F19FC1A3F1A0C1A4F1A1C1A5F1A2C1FF
:10092000A6F1A3C1A7F1A4C1A8F1A5C1A9F1A6C1CF
:10093000AAF1A7C1ABF1A8C1ACF1A9C1ADF1AAC19F
:10094000AEF1ABC1AFF1ACC1B0F1ADC1B1F1AEC16F
:10095000B2F1AFC1B3F1B0C1B4F1B1C1B5F1B2C13F
:10096000B6F1B3C1B7F1B4C1B8F1B5C1B9F1010184
:100970005E6B5F6B606B616B9A515E279B515F236F
:100980009C5160239D5161239E515E279F515F239F
:10099000A0516023A1516123A2515E27A3515F237F
:1009A000A4516023A5516123A6515E27A7515F235F
:1009B000A8516023A9516123AA515E27AB515F233F
:1009C000AC516023AD516123AE515E27AF515F231F
:1009D000B0516023B1516123B2515E27B3515F23FF
:1009E000B4516023B5516123B6515E27B7515F23DF
:1009F000B8516023B9516123D8900101613360334C
:100A00005F335E33D8900101613360335F335E330F
:100A1000D8900101613360335F335E3300C10CF164
:100A200001C10DF102C10EF103C10FF104C110F1BA
:100A300005C111F106C112F107C113F108C114F18A
:100A400009C115F10AC116F10BC117F134C135F115
:100A500011B836EF05F00101620E046F010E056F4B
:100A6000000E066F000E076F3FEF05F00101A70EA5
:100A7000046F020E056F000E066F000E076F5EC159
:100A800000F15FC101F160C102F161C103F1F0EC5D
:100A90002CF003BF04D01ABE02D01AA0108C11A0F3
:100AA00057EF05F010BA57EF05F00F80108A0CC110
:100AB00000F10DC101F10EC102F10FC103F110C12E
:100AC00004F111C105F112C106F113C107F114C1FE
:100AD00008F115C109F116C10AF117C10BF135C1B1
:100AE00034F113EF0BF00392ABB2AB98AB88030178
:100AF00003EE00F080517F0BE92604C0EFFF802B4E
:100B00008151805D700BD8A48B8200008051815D83
:100B1000700BD8A48B9281518019D8B4079013EF31
:100B20000BF0F2940101453F13EF0BF0462B13EF4E
:100B30000BF09E900101533F13EF0BF0542B13EF7A
:100B40000BF09E9211B82BEF08F0040066A1A9EFFC
:100B500005F08BB4B3EF05F010ACB3EF05F08B8468
:100B6000109CB4EF05F08B94077C07ACCFEF05F039
:100B7000C274C2B4C9EF05F0C3CFB7F5C4CFB8F59E
:100B80000501D890B833B733D890B833B733D0EF26
:100B900005F0C3CF55F1C4CF56F1D0EF05F0C282B6
:100BA00007B442EF06F047C14BF148C14CF149C1CF
:100BB0004DF14AC14EF15EC162F15FC163F160C1A6
:100BC00064F161C165F113A8E8EF05F0138C139887
:100BD0009AC1BAF19BC1BBF19CC1BCF19DC1BDF1F1
:100BE0009EC1BEF19FC1BFF1A0C1C0F1A1C1C1F1C1
:100BF000A2C1C2F1A3C1C3F1A4C1C4F1A5C1C5F191
:100C0000A6C1C6F1A7C1C7F1A8C1C8F1A9C1C9F160
:100C1000AAC1CAF1ABC1CBF1ACC1CCF1ADC1CDF130
:100C2000AEC1CEF1AFC1CFF1B0C1D0F1B1C1D1F100
:100C3000B2C1D2F1B3C1D3F1B4C1D4F1B5C1D5F1D0
:100C4000B6C1D6F1B7C1D7F1B8C1D8F1B9C1D9F1A0
:100C5000B7C5B9F5B8C5BAF5B9C5BBF5BAC5BCF5E0
:100C6000010155515B2756515C23E86A5D230E2E26
:100C700042EF06F05CC157F15DC158F15B6B5C6BF4
:100C80005D6B078E0201002F13EF0BF03C0E006F1F
:100C90001B50E00BE00AE866128819BE02D019B4B6
:100CA000108E00C10CF101C10DF102C10EF103C1A2
:100CB0000FF104C110F105C111F106C112F107C114
:100CC00013F108C114F109C115F10AC116F10BC1E4
:100CD00017F134C135F181AA23EF07F035A0F3EF06
:100CE00006F005012F51000AD8B423EF07F00501E3
:100CF0002F51010AD8B4ACEF06F005012F51020ABA
:100D0000D8B4EDEF06F005012F51030AD8B4EDEF8A
:100D100006F005012F51040AD8B4EDEF06F00501E5
:100D20002F51050AD8B4EDEF06F005012F51060A40
:100D3000D8B4EDEF06F005012F51070AD8B4EDEF56
:100D400006F005012F51320AD8B4AAEF06F02F6B36
:100D500023EF07F023EF07F005015767B7EF06F021
:100D60005867B7EF06F05967B7EF06F05A67BBEF61
:100D700006F023EF07F05BC500F15CC501F15DC52E
:100D800002F15EC503F10101010E046F000E056F53
:100D9000000E066F000E076FF0EC2CF000C15BF543
:100DA00001C15CF502C15DF503C15EF50067E0EFCE
:100DB00006F00167E0EF06F00267E0EF06F0036778
:100DC00023EF07F057C55BF558C55CF559C55DF5D0
:100DD0005AC55EF50F8823EF07F005013067F3EF82
:100DE00006F023EF07F00FBE08EF07F010A00DEF9D
:100DF00007F00101476704EF07F0486704EF07F0C9
:100E0000496704EF07F04A6708EF07F00DEF07F0B6
:100E100007AE0DEF07F020EF07F00501312F23EFAC
:100E200007F03C0E316F302F23EF07F00101000E69
:100E3000626FE00E636FA50E646F010E656F13881D
:100E40000501306B0F880501666B37B729EF07F096
:100E500066810CC100F10DC101F10EC102F10FC19B
:100E600003F110C104F111C105F112C106F113C162
:100E700007F114C108F115C109F116C10AF117C132
:100E80000BF135C134F100C10CF101C10DF102C10A
:100E90000EF103C10FF104C110F105C111F106C13A
:100EA00012F107C113F108C114F109C115F10AC10A
:100EB00016F10BC117F134C135F101018E6768EFEE
:100EC00007F08F6768EF07F0906768EF07F09167AA
:100ED0006CEF07F09CEF07F092C100F193C101F1B4
:100EE00094C102F195C103F10101010E046F000EDE
:100EF000056F000E066F000E076FF0EC2CF000C1BE
:100F000092F101C193F102C194F103C195F100671F
:100F100091EF07F0016791EF07F0026791EF07F09B
:100F200003679CEF07F08EC192F18FC193F190C1DE
:100F300094F191C195F10F80D57ED5BE6ED0D6CFFC
:100F400047F1D7CF48F145C149F1E86AE8CF4AF106
:100F5000138A1ABE02D01AA0108C109047C100F15B
:100F600048C101F149C102F14AC103F101010A0E70
:100F7000046F000E056F000E066F000E076FF0EC99
:100F80002CF003AF1080010154A7D3EF07F00F9AA4
:100F90000F9C0F9E0101000E5E6F600E5F6F3D0E95
:100FA000606F080E616F010147BFE3EF07F048670C
:100FB000E3EF07F04967E3EF07F04A67E3EF07F075
:100FC000F28808EF08F0F2985E6B5F6B606B616B04
:100FD0009A6B9B6B9C6B9D6B9E6B9F6BA06BA16BCD
:100FE000A26BA36BA46BA56BA66BA76BA86BA96B7D
:100FF000AA6BAB6BAC6BAD6BAE6BAF6BB06BB16B2D
:10100000B26BB36BB46BB56BB66BB76BB86BB96BDC
:10101000D76AD66A0101456B466B0CC100F10DC160
:1010200001F10EC102F10FC103F110C104F111C1B0
:1010300005F112C106F113C107F114C108F115C180
:1010400009F116C10AF117C10BF135C134F113EFE3
:101050000BF013EF0BF00201002F77EF0AF0D59E93
:10106000D6CF47F1D7CF48F145C149F1E86AE8CF7B
:101070004AF1138AD76AD66A0101456B466BD58E51
:101080001B50E00BE00AE866128819BE02D019B4C2
:10109000108E18AE1D8C00C10CF101C10DF102C102
:1010A0000EF103C10FF104C110F105C111F106C128
:1010B00012F107C113F108C114F109C115F10AC1F8
:1010C00016F10BC117F134C135F10FA0109A11B808
:1010D00075EF08F00101620E046F010E056F000E3E
:1010E000066F000E076F7EEF08F00101A70E046F78
:1010F000020E056F000E066F000E076F47C100F16C
:1011000048C101F149C102F14AC103F1F0EC2CF0F0
:1011100003BF91EF08F01ABE02D01AA0108C11B0D4
:101120000F800CC100F10DC101F10EC102F10FC120
:1011300003F110C104F111C105F112C106F113C18F
:1011400007F114C108F115C109F116C10AF117C15F
:101150000BF135C134F102013C0E006F00C10CF1FE
:1011600001C10DF102C10EF103C10FF104C110F173
:1011700005C111F106C112F107C113F108C114F143
:1011800009C115F10AC116F10BC117F134C135F1CE
:1011900081AA80EF09F035A050EF09F005012F5129
:1011A000000AD8B480EF09F005012F51010AD8B424
:1011B00009EF09F005012F51020AD8B44AEF09F0EE
:1011C00005012F51030AD8B44AEF09F005012F5148
:1011D000040AD8B44AEF09F005012F51050AD8B422
:1011E0004AEF09F005012F51060AD8B44AEF09F079
:1011F00005012F51070AD8B44AEF09F005012F5114
:10120000320AD8B407EF09F02F6B80EF09F080EFB6
:1012100009F00501576714EF09F0586714EF09F05A
:10122000596714EF09F05A6718EF09F080EF09F0D9
:101230005BC500F15CC501F15DC502F15EC503F15E
:101240000101010E046F000E056F000E066F000E07
:10125000076FF0EC2CF000C15BF501C15CF502C139
:101260005DF503C15EF500673DEF09F001673DEFF5
:1012700009F002673DEF09F0036780EF09F057C5F9
:101280005BF558C55CF559C55DF55AC55EF50F8827
:1012900080EF09F00501306750EF09F080EF09F0A9
:1012A0000FBE65EF09F010A06AEF09F00101476772
:1012B00061EF09F0486761EF09F0496761EF09F0F4
:1012C0004A6765EF09F06AEF09F007AE6AEF09F0C7
:1012D0007DEF09F00501312F80EF09F03C0E316FF1
:1012E000302F80EF09F00101000E626FE00E636F96
:1012F000A50E646F010E656F13880501306B0F88B2
:101300000501666B37B786EF09F066810CC100F105
:101310000DC101F10EC102F10FC103F110C104F1C1
:1013200011C105F112C106F113C107F114C108F191
:1013300015C109F116C10AF117C10BF135C134F11C
:1013400000C10CF101C10DF102C10EF103C10FF199
:1013500004C110F105C111F106C112F107C113F169
:1013600008C114F109C115F10AC116F10BC117F139
:1013700034C135F101018E67C5EF09F08F67C5EF04
:1013800009F09067C5EF09F09167C9EF09F0F9EF2F
:1013900009F092C100F193C101F194C102F195C12C
:1013A00003F10101010E046F000E056F000E066FC0
:1013B000000E076FF0EC2CF000C192F101C193F127
:1013C00002C194F103C195F10067EEEF09F00167E6
:1013D000EEEF09F00267EEEF09F00367F9EF09F0AD
:1013E0008EC192F18FC193F190C194F191C195F1A9
:1013F0000F80109047C100F148C101F149C102F1CD
:101400004AC103F101010A0E046F000E056F000EC0
:10141000066F000E076FF0EC2CF003AF1080010197
:1014200054A71FEF0AF00F9A0F9C0F9E0101000EA8
:101430005E6F600E5F6F3D0E606F080E616F47C19B
:1014400000F148C101F149C102F14AC103F10101B2
:10145000140E046F050E056F000E066F000E076F69
:10146000F0EC2CF003AF38EF0AF0F2885DEF0AF0F1
:10147000F2985E6B5F6B606B616B9A6B9B6B9C6BA6
:101480009D6B9E6B9F6BA06BA16BA26BA36BA46B00
:10149000A56BA66BA76BA86BA96BAA6BAB6BAC6BB0
:1014A000AD6BAE6BAF6BB06BB16BB26BB36BB46B60
:1014B000B56BB66BB76BB86BB96B0CC100F10DC1F6
:1014C00001F10EC102F10FC103F110C104F111C10C
:1014D00005F112C106F113C107F114C108F115C1DC
:1014E00009F116C10AF117C10BF135C134F104003D
:1014F0008BB482EF0AF010AC82EF0AF08B84109C60
:1015000083EF0AF08B94077C07AC9EEF0AF0C2745D
:10151000C2B498EF0AF0C3CFB7F5C4CFB8F5050150
:10152000D890B833B733D890B833B7339FEF0AF0B9
:10153000C3CF55F1C4CF56F19FEF0AF0C28207B472
:1015400011EF0BF047C14BF148C14CF149C14DF1CE
:101550004AC14EF15EC162F15FC163F160C164F1E5
:1015600061C165F113A8B7EF0AF0138C13989AC103
:10157000BAF19BC1BBF19CC1BCF19DC1BDF19EC143
:10158000BEF19FC1BFF1A0C1C0F1A1C1C1F1A2C113
:10159000C2F1A3C1C3F1A4C1C4F1A5C1C5F1A6C1E3
:1015A000C6F1A7C1C7F1A8C1C8F1A9C1C9F1AAC1B3
:1015B000CAF1ABC1CBF1ACC1CCF1ADC1CDF1AEC183
:1015C000CEF1AFC1CFF1B0C1D0F1B1C1D1F1B2C153
:1015D000D2F1B3C1D3F1B4C1D4F1B5C1D5F1B6C123
:1015E000D6F1B7C1D7F1B8C1D8F1B9C1D9F1B7C5F2
:1015F000B9F5B8C5BAF5B9C5BBF5BAC5BCF50101B1
:1016000055515B2756515C23E86A5D230E2E11EF7E
:101610000BF05CC157F15DC158F15B6B5C6B5D6BAE
:10162000078E13EF0BF002C0E0FF005001C0D8FF9F
:101630001000A6B219EF0BF00CC0A9FF0BC0A8FF59
:10164000A69EA69CA684F29E550EA76EAA0EA76E15
:10165000A682F28EA694A6B22BEF0BF00C2A1200F3
:10166000A96EA69EA69CA680A8500C2A1200040172
:101670002C0E826F8CEC0EF0EBEC2DF00C5030EC5D
:101680000BF0E8CF00F10C5030EC0BF0E8CF01F19B
:1016900001AF50EF0BF00101FF0E026FFF0E036F61
:1016A0008EEC2DF029675CEF0BF00401200E826FA9
:1016B0008CEC0EF061EF0BF004012D0E826F8CECC0
:1016C0000EF098EC2BF01200356A076A0F6A106A68
:1016D000116A126A136A0F010D0EC16E860EC06E7A
:1016E000030EC26E0F01680E896E130E926E080E05
:1016F0008A6EF30E936E8B6A900E946EC80E30EC69
:101700000BF0E8CFE8FF1098E8A0108810A805D0EB
:101710000E0E236E8E0E246E04D00F0E236E8F0ECF
:10172000246E6AEC2EF0F18EF19EFC0E30EC0BF084
:10173000E8CF0BF00BA011800BA211820BA4118437
:101740000BA81188C90E30EC0BF0E8CF18F0CA0EC8
:1017500030EC0BF0E8CF19F0CB0E30EC0BF0E8CF0B
:101760001AF0CC0E30EC0BF0E8CF1BF0CE0E30ECC4
:101770000BF0E8CF14F0CD0E30EC0BF0E8CF34F0E6
:101780001D6A1E6A0E6A01015B6B5C6B5D6B576BB9
:10179000586BF29A0101476B486B496B4A6B4B6B74
:1017A0004C6B4D6B4E6B4F6B506B516B526B456B73
:1017B000466BD76AD66A0F01280ED56EF28A9D90C5
:1017C000B00ECD6E01015E6B5F6B606B616B626B27
:1017D000636B646B656B666B676B686B696B536B94
:1017E000546BCF6ACE6A0F9A0F9C0F9E9D80760E27
:1017F000CA6E9D8202013C0E006FCC6A160E30EC60
:101800000BF0E8CF00F1170E30EC0BF0E8CF01F150
:10181000180E30EC0BF0E8CF02F1190E30EC0BF0A3
:10182000E8CF03F1010103AF30EF0CF0EBEC2DF04A
:10183000160E0C6E00C10BF019EC0BF0170E0C6EAF
:1018400001C10BF019EC0BF0180E0C6E02C10BF07D
:1018500019EC0BF0190E0C6E03C10BF019EC0BF028
:1018600000C18EF101C18FF102C190F103C191F16C
:1018700000C192F101C193F102C194F103C195F14C
:101880001A0E30EC0BF0E8CF00F11B0E30EC0BF031
:10189000E8CF01F11C0E30EC0BF0E8CF02F11D0E89
:1018A00030EC0BF0E8CF03F1010103AF86EF0CF051
:1018B000EBEC2DF01A0E0C6E00C10BF019EC0BF0D6
:1018C0001B0E0C6E01C10BF019EC0BF01C0E0C6E14
:1018D00002C10BF019EC0BF01D0E0C6E03C10BF0E6
:1018E00019EC0BF01A0E30EC0BF0E8CF00F11B0EE8
:1018F00030EC0BF0E8CF01F11C0E30EC0BF0E8CF30
:1019000002F11D0E30EC0BF0E8CF03F100C196F1AF
:1019100001C197F102C198F103C199F1240EAC6E97
:10192000900EAB6E240EAC6E080EB86E000EB06E4C
:101930001F0EAF6E0401806B816B0F01900EAB6EBA
:101940000F019D8A0301806B816BC26B8B920EEC41
:1019500033F00EEC33F06CEC34F0EDEC30F0200EA4
:1019600030EC0BF0E8CF2FF505012F51FF0AD8A47A
:10197000C1EF0CF02F6B200E0C6E2FC50BF019EC85
:101980000BF00501010E306F3C0E316F250E30EC6F
:101990000BF0E8CF00F1260E30EC0BF0E8CF01F1B0
:1019A000270E30EC0BF0E8CF02F1280E30EC0BF0F4
:1019B000E8CF03F1010103AFF8EF0CF0EBEC2DF0F1
:1019C000250E0C6E00C10BF019EC0BF0260E0C6E00
:1019D00001C10BF019EC0BF0270E0C6E02C10BF0DD
:1019E00019EC0BF0280E0C6E03C10BF019EC0BF088
:1019F00000C157F501C158F502C159F503C15AF5A7
:101A000000C15BF501C15CF502C15DF503C15EF586
:101A1000290E30EC0BF0E8CF5FF5050160515F5DFA
:101A2000D8A05FC560F5210E30EC0BF0E8CF00F1D7
:101A3000220E30EC0BF0E8CF01F1230E30EC0BF06E
:101A4000E8CF02F1240E30EC0BF0E8CF03F10101F6
:101A500003AF59EF0DF0EBEC2DF0210E0C6E00C131
:101A60000BF019EC0BF0220E0C6E01C10BF019EC0F
:101A70000BF0230E0C6E02C10BF019EC0BF0240ED0
:101A80000C6E03C10BF019EC0BF0210E30EC0BF0D7
:101A9000E8CF00F1220E30EC0BF0E8CF01F1230E7D
:101AA00030EC0BF0E8CF02F1240E30EC0BF0E8CF75
:101AB00003F100C161F501C162F502C163F503C123
:101AC00064F535EC30F01BEC2FF073EC2EF035A004
:101AD000CAEF0DF005012F51020A16E005012F5142
:101AE000030A19E005012F51040A24E005012F51D2
:101AF000050A2BE005012F51060A39E005012F5197
:101B0000070A3FE0CAEF0DF0602FC7EF0DF05FC589
:101B100060F5CAEF0DF0B0C500F101010F0E00171E
:101B200001010051000A36E001010051050A32E0CE
:101B3000C7EF0DF0B0C500F101010F0E0017010154
:101B40000051000A27E0C7EF0DF00501B051000A6F
:101B500021E00501B051150A1DE00501B051300A20
:101B600019E00501B051450A15E0C7EF0DF0050178
:101B7000B051000A0FE00501B051300A0BE0C7EF89
:101B80000DF00501B051000A05E0C7EF0DF081BA74
:101B9000ABEF34F007900001F28EF28C12AE03D05E
:101BA00012BCD7EF18F007B01EEF2AF00FB031EFDC
:101BB00023F010BE31EF23F012B831EF23F00FB84D
:101BC000BFEF1CF00301805181197F0BD8B41EEFC9
:101BD0002AF013EE00F081517F0BE126812BE7CF35
:101BE000E8FFE00BD8B41EEF2AF023EE82F0C251DA
:101BF0003F0BD926E7CFDFFFC22BDF50780AD8A4EE
:101C00001EEF2AF0078092C100F193C101F194C147
:101C100002F195C103F10101040E046F000E056F7E
:101C2000000E066F000E076FF0EC2CF000AF22EFF5
:101C30000EF00101030E926F000E936F000E946F71
:101C4000000E956F03018251720AD8B40DEF23F094
:101C50008251520AD8B40DEF23F08251750AD8B4DC
:101C60000DEF23F08251680AD8B4A0EF0EF0825134
:101C7000630AD8B4D8EF26F08251690AD8B4B7EF16
:101C80001FF082517A0AD8B4CAEF20F08251490A73
:101C9000D8B456EF1FF08251500AD8B474EF1EF03A
:101CA0008251700AD8B4B7EF1EF08251540AD8B4EA
:101CB000E2EF1EF08251740AD8B428EF1FF082516F
:101CC000410AD8B4A4EF0FF082514B0AD8B4A2EF66
:101CD0000EF082516D0AD8B4E1EF13F082514D0A33
:101CE000D8B4FAEF13F08251730AD8B43DEF22F062
:101CF0008251530AD8B4A2EF22F082514C0AD8B4D0
:101D000089EF14F08251590AD8B432EF13F012AEB1
:101D100001D0128C0FEF27F0040114EE00F0805177
:101D20007F0BE12682C4E7FF802B120004010D0E19
:101D3000826F8CEC0EF00A0E826F8CEC0EF01200AB
:101D40000DEF27F004014B0E826F8CEC0EF00401B6
:101D50002C0E826F8CEC0EF081B802D034B630D0ED
:101D600003018351430AD8B4E7EF0EF00301835116
:101D7000630AD8B4E9EF0EF003018351520AD8B4D4
:101D8000EBEF0EF003018351720AD8B4EDEF0EF0C1
:101D900003018351470AD8B4EFEF0EF003018351DA
:101DA000670AD8B4F1EF0EF003018351540AD8B496
:101DB000F3EF0EF003018351740AD8B462EF0FF011
:101DC00003018351550AD8B4F5EF0EF082D0348068
:101DD0007AD0349078D0348276D0349274D03484EF
:101DE00072D0349470D034866ED084C330F185C301
:101DF00031F186C332F187C333F10101296B39EC2C
:101E00002EF0B0EC2DF000C104F101C105F102C1CA
:101E100006F103C107F12CEC2EF0200EF86EF76AE4
:101E2000F66A0900F5CF2CF10900F5CF2DF1090074
:101E3000F5CF2EF10900F5CF2FF10900F5CF30F1E4
:101E40000900F5CF31F10900F5CF32F10900F5CFE6
:101E500033F10101296B39EC2EF0B0EC2DF0F0ECF0
:101E60002CF000673BEF0FF001673BEF0FF00267CC
:101E70003BEF0FF0036701D025D004014E0E826FB7
:101E80008CEC0EF004016F0E826F8CEC0EF00401EE
:101E90004D0E826F8CEC0EF00401610E826F8CECA3
:101EA0000EF00401740E826F8CEC0EF00401630ED0
:101EB000826F8CEC0EF00401680E826F8CEC0EF0D9
:101EC0000DEF27F03496CD0E0C6E34C00BF019ECEC
:101ED0000BF0CD0E30EC0BF0E8CF34F034B006D080
:101EE0000401630E826F8CEC0EF005D00401430EEA
:101EF000826F8CEC0EF034B206D00401720E826F49
:101F00008CEC0EF005D00401520E826F8CEC0EF0BA
:101F100034B406D00401670E826F8CEC0EF005D04D
:101F20000401470E826F8CEC0EF034B606D004012B
:101F3000740E826F8CEC0EF005D00401540E826F8B
:101F40008CEC0EF00DEF27F00401410E826F8CEC4B
:101F50000EF003018351310AD8B452EF12F003019D
:101F60008351320AD8B482EF11F003018351330A4E
:101F7000D8B40BEF11F003018351340AD8B4FBEF4E
:101F80000FF003018351350AD8B4CEEF0FF00401EE
:101F90003F0E826F8CEC0EF00DEF27F003018451A1
:101FA000300AD8B4DCEF0FF003018451310AD8B401
:101FB000DFEF0FF0E0EF0FF08B90E0EF0FF08B8092
:101FC0000401350E826F8CEC0EF004012C0E826F32
:101FD0008CEC0EF08BB0F4EF0FF00401300E826F3A
:101FE0008CEC0EF0F9EF0FF00401310E826F8CECE7
:101FF0000EF00DEF27F0CC0E30EC0BF0E8CF0BF02D
:1020000004012C0E826F8CEC0EF003018451310A16
:10201000D8B41FEF10F003018451300AD8B421EF77
:1020200010F0030184514D0AD8B42BEF10F00301D6
:102030008451540AD8B432EF10F049EF10F08A847A
:1020400001D08A940BAE04D00BAC02D00BBA21D0D5
:10205000E00E0B1218D01F0E0B168539E844E00B6A
:102060000B1211D0E00E0B162CEC2EF085C332F1C2
:1020700086C333F10101296B39EC2EF0B0EC2DF061
:1020800000511F0B0B12CC0E0C6E0BC00BF019EC99
:102090000BF00401340E826F8CEC0EF004012C0E58
:1020A000826F8CEC0EF0CC0E30EC0BF0E8CF1BF016
:1020B0008AB406D00401300E826F8CEC0EF005D08D
:1020C0000401310E826F8CEC0EF004012C0E826F35
:1020D0008CEC0EF01B38E840070BE8CF82F40401CB
:1020E000300E82278CEC0EF004012C0E826F8CECEB
:1020F0000EF0EBEC2DF01B501F0BE8CF00F18EEC37
:102100002DF032C182F40401300E82278CEC0EF0E7
:1021100033C182F40401300E82278CEC0EF00401EE
:102120002C0E826F8CEC0EF0EBEC2DF02EC000F13B
:1021300000AF0BD0FF0E016FFF0E026FFF0E036F9B
:1021400004012D0E826F8CEC0EF08EEC2DF031C15F
:1021500082F40401300E82278CEC0EF032C182F43E
:102160000401300E82278CEC0EF033C182F404019E
:10217000300E82278CEC0EF004012C0E826F8CEC5A
:102180000EF0EBEC2DF02DC000F18EEC2DF031C1F6
:1021900082F40401300E82278CEC0EF032C182F4FE
:1021A0000401300E82278CEC0EF033C182F404015E
:1021B000300E82278CEC0EF004012C0E826F8CEC1A
:1021C0000EF0EBEC2DF02FC000F100AF0BD0FF0EA6
:1021D000016FFF0E026FFF0E036F04012D0E826F61
:1021E0008CEC0EF08EEC2DF031C182F40401300E37
:1021F00082278CEC0EF032C182F40401300E82276B
:102200008CEC0EF033C182F40401300E82278CEC8A
:102210000EF00DEF27F0CB0E30EC0BF0E8CF0BF00B
:1022200004012C0E826F8CEC0EF003018451450AE0
:10223000D8B42FEF11F003018451440AD8B432EF1F
:1022400011F003018451300AD8B435EF11F00301C5
:102250008451310AD8B439EF11F044EF11F00B9EDC
:102260003EEF11F00B8E3EEF11F0FC0E0B163EEF21
:1022700011F0FC0E0B160B803EEF11F0CB0E0C6E26
:102280000BC00BF019EC0BF00401330E826F8CECD9
:102290000EF004012C0E826F8CEC0EF0CB0E30ECA5
:1022A0000BF0E8CF1AF01ABE5DEF11F00401450EF5
:1022B000826F8CEC0EF062EF11F00401440E826F1D
:1022C0008CEC0EF004012C0E826F8CEC0EF00401ED
:1022D000300E826F8CEC0EF004012C0E826F8CECB1
:1022E0000EF01AB07BEF11F00401300E826F8CEC0F
:1022F0000EF080EF11F00401310E826F8CEC0EF0C5
:102300000DEF27F0CA0E30EC0BF0E8CF0BF0040114
:102310002C0E826F8CEC0EF003018451450AD8B468
:10232000BEEF11F003018451440AD8B4C1EF11F09B
:10233000030184514D0AD8B4CAEF11F0030184514E
:10234000410AD8B4C4EF11F003018451460AD8B44D
:10235000C7EF11F003018451560AD8B4D2EF11F03F
:1023600003018451500AD8B4DDEF11F00301845108
:10237000520AD8B4E0EF11F0E9EF11F00B9EE3EF51
:1023800011F00B8EE3EF11F00B9CE3EF11F00B8CCF
:10239000E3EF11F0FC0E0B1685C3E8FF030B0B12E5
:1023A000E3EF11F0C70E0B1685C3E8FF070BE846F5
:1023B000E846E8460B12E3EF11F00B84E3EF11F06F
:1023C0000B94E3EF11F0CA0E0C6E0BC00BF019EC7E
:1023D0000BF0CA0E30EC0BF0E8CF19F00401320E0E
:1023E000826F8CEC0EF004012C0E826F8CEC0EF0E0
:1023F00019BE02EF12F00401450E826F8CEC0EF054
:1024000007EF12F00401440E826F8CEC0EF0040111
:102410002C0E826F8CEC0EF019C0E8FF030BE8CF96
:1024200082F40401300E82278CEC0EF004012C0E95
:10243000826F8CEC0EF019BC25EF12F00401410EF6
:10244000826F8CEC0EF02AEF12F00401460E826FC0
:102450008CEC0EF004012C0E826F8CEC0EF019C087
:10246000E8FF380BE842E842E842E8CF82F4040192
:10247000300E82278CEC0EF004012C0E826F8CEC57
:102480000EF019B44BEF12F00401520E826F8CEC77
:102490000EF050EF12F00401500E826F8CEC0EF033
:1024A0000DEF27F0C90E30EC0BF0E8CF0BF0040174
:1024B0002C0E826F8CEC0EF003018451450AD8B4C7
:1024C00070EF12F003018451440AD8B473EF12F094
:1024D000030184514D0AD8B476EF12F084EF12F064
:1024E0000B9E7EEF12F00B8E7EEF12F0F80E0B16A5
:1024F00085C3E8FF070B0B127EEF12F0C90E0C6EBE
:102500000BC00BF019EC0BF00401310E826F8CEC58
:102510000EF004012C0E826F8CEC0EF0C90E30EC24
:102520000BF0E8CF18F018BE06D00401450E826FFC
:102530008CEC0EF005D00401440E826F8CEC0EF092
:1025400004012C0E826F8CEC0EF018C0E8FF070B14
:10255000E8CF82F40401300E82278CEC0EF00401E7
:102560002C0E826F8CEC0EF00780EBEC2DF029C066
:10257000E8FF003B00430043030B8EEC2DF033C11A
:1025800082F40401300E82278CEC0EF004012C0E34
:10259000826F8CEC0EF0EBEC2DF029C001F1019F65
:1025A000019D2AC000F101018EEC2DF02FC182F4B3
:1025B0000401300E82278CEC0EF030C182F404014D
:1025C000300E82278CEC0EF031C182F40401300E03
:1025D00082278CEC0EF032C182F40401300E822787
:1025E0008CEC0EF033C182F40401300E82278CECA7
:1025F0000EF004012C0E826F8CEC0EF0EBEC2DF043
:102600002BC001F12CC000F1D89001330033D890D9
:102610000133003301018EEC2DF02FC182F404014F
:10262000300E82278CEC0EF030C182F40401300EA3
:1026300082278CEC0EF031C182F40401300E822727
:102640008CEC0EF032C182F40401300E82278CEC47
:102650000EF033C182F40401300E82278CEC0EF0B0
:102660000DEF27F0FC0E30EC0BF0E8CF0BF0030180
:102670008351520AD8B469EF13F003018351720AEF
:10268000D8B46CEF13F003018351500AD8B46FEF44
:1026900013F003018351700AD8B472EF13F00301F1
:1026A0008351550AD8B475EF13F003018351750AAD
:1026B000D8B478EF13F003018351430AD8B481EF03
:1026C00013F003018351630AD8B484EF13F08DEF44
:1026D00013F00B9087EF13F00B8087EF13F00B9242
:1026E00087EF13F00B8287EF13F00B9487EF13F053
:1026F0000B8487EF13F00B9687EF13F00B8687EFB1
:1027000013F00B9887EF13F00B8887EF13F0FC0E94
:102710000C6E0BC00BF019EC0BF00401590E826F1C
:102720008CEC0EF01190119211941198FC0E30EC7B
:102730000BF0E8CF0BF00BA011800BA211820BA4C1
:1027400011840BA8118811A0ADEF13F00401520EF3
:10275000826F8CEC0EF0B2EF13F00401720E826FF8
:102760008CEC0EF011A8BCEF13F00401430E826F45
:102770008CEC0EF0C1EF13F00401630E826F8CEC51
:102780000EF011A2CBEF13F00401500E826F8CEC0F
:102790000EF0D0EF13F00401700E826F8CEC0EF08F
:1027A00011A4DAEF13F00401550E826F8CEC0EF0D9
:1027B000DFEF13F00401750E826F8CEC0EF00DEF5D
:1027C00027F004016D0E826F8CEC0EF00301835133
:1027D000300AD8B439EF14F003018351310AD8B468
:1027E0004CEF14F003018351320AD8B45FEF14F0B8
:1027F0000FEF27F004014D0E826F8CEC0EF02CECE5
:102800002EF084C331F185C332F186C333F1010167
:10281000296B39EC2EF0B0EC2DF003018351300A16
:10282000D8B421EF14F003018351310AD8B429EF51
:1028300014F003018351320AD8B431EF14F00FEFD2
:1028400027F0FD0E0C6E00C10BF019EC0BF039EF08
:1028500014F0FE0E0C6E00C10BF019EC0BF04CEFF7
:1028600014F0FF0E0C6E00C10BF019EC0BF05FEFD3
:1028700014F00401300E826F8CEC0EF004012C0E6B
:10288000826F8CEC0EF0EBEC2DF0FD0E30EC0BF0CB
:10289000E8CF00F170EF14F00401310E826F8CEC80
:1028A0000EF004012C0E826F8CEC0EF0EBEC2DF090
:1028B000FE0E30EC0BF0E8CF00F170EF14F00401E5
:1028C000320E826F8CEC0EF0EBEC2DF004012C0E2E
:1028D000826F8CEC0EF0FF0E30EC0BF0E8CF00F1C5
:1028E0008EEC2DF031C182F40401300E82278CEC85
:1028F0000EF032C182F40401300E82278CEC0EF00F
:1029000033C182F40401300E82278CEC0EF00DEFFF
:1029100027F003018351300AD8B484EF19F0030182
:102920008351310AD8B4B1EF1AF003018351320A4E
:10293000D8B41FEF1BF003018351330AD8B42FEF33
:102940001BF003018351340AD8B43FEF1BF003019D
:102950008351350AD8B4C5EF1CF003018351360A00
:10296000D8B4F3EF1CF003018351370AD8B45CEFFD
:1029700017F003018351380AD8B4FAEF17F00301B6
:102980008351460AD8B418EF1CF0030183514D0A55
:10299000D8B4D5EF15F0030183516D0AD8B4EFEF29
:1029A00015F0030183515A0AD8B42BEF1AF0030132
:1029B0008351490AD8B4F3EF1DF003018351500A43
:1029C000D8B425EF1DF003018351540AD8B49EEF0B
:1029D0001DF003018351630AD8B40FEF16F0030111
:1029E0008351430AD8B407EF17F003018351730AE8
:1029F000D8B40DEF16F003018351610AD8B422EF69
:102A000015F003018351650AD8B4D4EF19F003011E
:102A10008351450AD8B4E2EF19F003018351620AE9
:102A2000D8B4F0EF19F003018351420AD8B4FEEF95
:102A300019F003018351760AD8B40CEF1AF0D8A428
:102A40000FEF27F004014C0E826F8CEC0EF00401A6
:102A5000610E826F8CEC0EF01BEC2FF004012C0E3B
:102A6000826F8CEC0EF0EBEC2DF0AFC500F10101A4
:102A70008EEC2DF031C182F40401300E82278CECF3
:102A80000EF032C182F40401300E82278CEC0EF07D
:102A900033C182F40401300E82278CEC0EF0040165
:102AA0002C0E826F8CEC0EF0EBEC2DF0B0C500F12B
:102AB00001018EEC2DF031C182F40401300E822729
:102AC0008CEC0EF032C182F40401300E82278CECC3
:102AD0000EF033C182F40401300E82278CEC0EF02C
:102AE00004012C0E826F8CEC0EF0EBEC2DF0B1C5D6
:102AF00000F101018EEC2DF031C182F40401300EA1
:102B000082278CEC0EF032C182F40401300E822751
:102B10008CEC0EF033C182F40401300E82278CEC71
:102B20000EF004012C0E826F8CEC0EF0EBEC2DF00D
:102B3000B2C500F101018EEC2DF031C182F4040127
:102B4000300E82278CEC0EF032C182F40401300E7C
:102B500082278CEC0EF033C182F40401300E822700
:102B60008CEC0EF004012C0E826F8CEC0EF0EBEC72
:102B70002DF0B6C500F101018EEC2DF031C182F4CB
:102B80000401300E82278CEC0EF032C182F4040175
:102B9000300E82278CEC0EF033C182F40401300E2B
:102BA00082278CEC0EF021EF1DF02CEC2EF084C36C
:102BB00033F139EC2EF0B0EC2DF0200E0C6E00C18C
:102BC0000BF019EC0BF000C12FF505012F51000A95
:102BD00006E005012F51010A02E0B5EC2FF00401D7
:102BE0004C0E826F8CEC0EF004014D0E826F8CEC5B
:102BF0000EF004012C0E826F8CEC0EF0EBEC2DF03D
:102C00002FC500F18EEC2DF033C182F40401300E9B
:102C100082278CEC0EF021EF1DF0ABEF34F00401B5
:102C20004C0E826F8CEC0EF00401630E826F8CEC04
:102C30000EF073EC2EF004012C0E826F8CEC0EF073
:102C400024EC16F021EF1DF0EBEC2DF0B5C500F1F2
:102C50000101003B0F0E00178EEC2DF033C182F402
:102C60000401300E82278CEC0EF0B5C500F1010195
:102C70000F0E010100178EEC2DF033C182F4040118
:102C8000300E82278CEC0EF004012D0E826F8CEC3E
:102C90000EF0B4C500F10101003B0F0E00178EECE1
:102CA0002DF033C182F40401300E82278CEC0EF03B
:102CB000B4C500F101010F0E010100178EEC2DF0DB
:102CC00033C182F40401300E82278CEC0EF0040133
:102CD0002D0E826F8CEC0EF0B3C500F10101003BAC
:102CE0000F0E00178EEC2DF033C182F40401300E6C
:102CF00082278CEC0EF0B3C500F101010F0E01012B
:102D000000178EEC2DF033C182F40401300E8227BF
:102D10008CEC0EF00401200E826F8CEC0EF0B2C52C
:102D200000F10F0E010100178EEC2DF033C182F47B
:102D30000401300E82278CEC0EF00401200E826F0D
:102D40008CEC0EF0B1C500F101010101003B0F0E4A
:102D500000178EEC2DF033C182F40401300E82276F
:102D60008CEC0EF0B1C500F101010F0E010100174E
:102D70008EEC2DF033C182F40401300E82278CECEE
:102D80000EF004013A0E826F8CEC0EF0B0C500F12B
:102D90000101003B0F0E00178EEC2DF033C182F4C1
:102DA0000401300E82278CEC0EF0B0C500F1010159
:102DB0000F0E010100178EEC2DF033C182F40401D7
:102DC000300E82278CEC0EF004013A0E826F8CECF0
:102DD0000EF0AFC500F10101003B0F0E00178EECA5
:102DE0002DF033C182F40401300E82278CEC0EF0FA
:102DF000AFC500F101010F0E00178EEC2DF033C1AD
:102E000082F40401300E82278CEC0EF0120084C391
:102E1000E8FF0F0BE83AE8CFB5F585C3E8FF0F0BE5
:102E20000501B51387C3E8FF0F0BE83AE8CFB4F507
:102E300088C3E8FF0F0B0501B4138AC3E8FF0F0B2B
:102E4000E83AE8CFB3F58BC3E8FF0F0B0501B313E6
:102E50008DC3E8FF0F0BE8CFB2F58FC3E8FF0F0B70
:102E6000E83AE8CFB1F590C3E8FF0F0B0501B113C5
:102E700092C3E8FF0F0BE83AE8CFB0F593C3E8FF41
:102E80000F0B0501B01395C3E8FF0F0BE83AE8CF2D
:102E9000AFF596C3E8FF0F0B0501AF13CEEC2EF094
:102EA00004014C0E826F8CEC0EF00401430E826F15
:102EB0008CEC0EF019EF16F0078404014C0E826FB3
:102EC0008CEC0EF00401370E826F8CEC0EF00401D6
:102ED0002C0E826F8CEC0EF005012E51130A06E0C9
:102EE00005012E51170A0DE0F7EF17F00101000E52
:102EF000006F000E016F100E026F000E036F8AEF5D
:102F000017F00101000E006F000E016F000E026F3E
:102F1000010E036F8EEC2DF02AC182F40401300EF5
:102F200082278CEC0EF02BC182F40401300E822734
:102F30008CEC0EF02CC182F40401300E82278CEC54
:102F40000EF02DC182F40401300E82278CEC0EF0BD
:102F50002EC182F40401300E82278CEC0EF02FC1BA
:102F600082F40401300E82278CEC0EF030C182F422
:102F70000401300E82278CEC0EF031C182F4040182
:102F8000300E82278CEC0EF032C182F40401300E38
:102F900082278CEC0EF033C182F40401300E8227BC
:102FA0008CEC0EF004012C0E826F8CEC0EF0010103
:102FB000100E006F000E016F000E026F000E036F07
:102FC0008EEC2DF031C182F40401300E82278CEC9E
:102FD0000EF032C182F40401300E82278CEC0EF028
:102FE00033C182F40401300E82278CEC0EF007947A
:102FF00021EF1DF00501216B226B236B246B040173
:103000004C0E826F8CEC0EF00401380E826F8CEC4B
:103010000EF004012C0E826F8CEC0EF00101100EEC
:10302000006F000E016F000E026F000E036F8EEC3A
:103030002DF02AC182F40401300E82278CEC0EF0B0
:103040002BC182F40401300E82278CEC0EF02CC1CF
:1030500082F40401300E82278CEC0EF02DC182F434
:103060000401300E82278CEC0EF02EC182F4040194
:10307000300E82278CEC0EF02FC182F40401300E4A
:1030800082278CEC0EF030C182F40401300E8227CE
:103090008CEC0EF031C182F40401300E82278CECEE
:1030A0000EF032C182F40401300E82278CEC0EF057
:1030B00033C182F40401300E82278CEC0EF004013F
:1030C0002C0E826F8CEC0EF025C500F126C501F1A7
:1030D00027C502F128C503F10101100E046F000E8F
:1030E000056F000E066F000E076F21EC2DF000C17A
:1030F00033F501C134F502C135F503C136F58EEC67
:103100002DF02AC182F40401300E82278CEC0EF0DF
:103110002BC182F40401300E82278CEC0EF02CC1FE
:1031200082F40401300E82278CEC0EF02DC182F463
:103130000401300E82278CEC0EF02EC182F40401C3
:10314000300E82278CEC0EF02FC182F40401300E79
:1031500082278CEC0EF030C182F40401300E8227FD
:103160008CEC0EF031C182F40401300E82278CEC1D
:103170000EF032C182F40401300E82278CEC0EF086
:1031800033C182F40401300E82278CEC0EF096ECF1
:103190000EF005013367D4EF18F03467D4EF18F060
:1031A0003567D4EF18F0366702D073EF19F0129E2E
:1031B000129C21C500F122C501F123C502F124C5ED
:1031C00003F1899A400EC76E200EC66E9E96C69E6B
:1031D0000B0EC96EFF0E9EB602D0E82EFCD79E964F
:1031E000C69E02C1C9FFFF0E9EB602D0E82EFCD7D4
:1031F0009E96C69E01C1C9FFFF0E9EB602D0E82E64
:10320000FCD79E96C69E00C1C9FFFF0E9EB602D097
:10321000E82EFCD79E96C69EC952FF0E9EB602D0DF
:10322000E82EFCD70501100E326F040114EE00F0F9
:1032300080517F0BE1269E96C69EC952FF0E9EB618
:1032400002D0E82EFCD7C9CFE7FF0401802B05018F
:10325000322F15EF19F0898A33C500F134C501F119
:1032600035C502F136C503F10101010E046F000EF0
:10327000056F000E066F000E076FF0EC2CF000C11A
:1032800033F501C134F502C135F503C136F5050149
:10329000336752EF19F0346752EF19F0356752EF88
:1032A00019F0366702D073EF19F021C500F122C57D
:1032B00001F123C502F124C503F10101100E046FD1
:1032C000000E056F000E066F000E076FF5EC2CF078
:1032D00000C121F501C122F502C123F503C124F586
:1032E000128E0FEF27F00401450E826F8CEC0EF06A
:1032F00004014F0E826F8CEC0EF00401460E826FBB
:103300008CEC0EF021EF1DF007846CEC34F0EBEC4C
:103310002DF02DC500F18EEC2DF004014C0E826FC6
:103320008CEC0EF00401300E826F8CEC0EF0040178
:103330002C0E826F8CEC0EF031C182F40401300E41
:1033400082278CEC0EF032C182F40401300E822709
:103350008CEC0EF033C182F40401300E82278CEC29
:103360000EF004012C0E826F8CEC0EF0EBEC2DF0C5
:103370002EC500F18EEC2DF031C182F40401300E27
:1033800082278CEC0EF032C182F40401300E8227C9
:103390008CEC0EF033C182F40401300E82278CECE9
:1033A0000EF0079421EF1DF004014C0E826F8CEC9F
:1033B0000EF00401650E826F8CEC0EF091EC30F093
:1033C00021EF1DF004014C0E826F8CEC0EF0040115
:1033D000450E826F8CEC0EF0A8EC30F021EF1DF062
:1033E00004014C0E826F8CEC0EF00401620E826FB1
:1033F0008CEC0EF0D6EC30F021EF1DF004014C0EF9
:10340000826F8CEC0EF00401420E826F8CEC0EF099
:10341000BFEC30F021EF1DF004014C0E826F8CECFC
:103420000EF00401760E826F8CEC0EF004012C0E6F
:10343000826F8CEC0EF010A807D00401310E826F61
:103440008CEC0EF021EF1DF00401300E826F8CEC3D
:103450000EF021EF1DF004014C0E826F8CEC0EF08B
:1034600004015A0E826F8CEC0EF004012C0E826F58
:103470008CEC0EF06CEC34F0EBEC2DF005012E51E1
:10348000130A06E005012E51170A0DE05CEF1AF051
:103490000101000E006F000E016F100E026F000E92
:1034A000036F5CEF1AF00101000E006F000E016F58
:1034B000000E026F010E036F0101100E046F000E6B
:1034C000056F000E066F000E076F21EC2DF08EECDD
:1034D0002DF02AC182F40401300E82278CEC0EF00C
:1034E0002BC182F40401300E82278CEC0EF02CC12B
:1034F00082F40401300E82278CEC0EF02DC182F490
:103500000401300E82278CEC0EF02EC182F40401EF
:10351000300E82278CEC0EF02FC182F40401300EA5
:1035200082278CEC0EF030C182F40401300E822729
:103530008CEC0EF031C182F40401300E82278CEC49
:103540000EF032C182F40401300E82278CEC0EF0B2
:1035500033C182F40401300E82278CEC0EF021EF8F
:103560001DF0078404014C0E826F8CEC0EF00401F8
:10357000310E826F8CEC0EF004012C0E826F8CECFD
:103580000EF025C500F126C501F127C502F128C5B9
:1035900003F10101100E046F000E056F000E066F9F
:1035A000000E076F21EC2DF08EEC2DF02AC182F475
:1035B0000401300E82278CEC0EF02BC182F4040142
:1035C000300E82278CEC0EF02CC182F40401300EF8
:1035D00082278CEC0EF02DC182F40401300E82277C
:1035E0008CEC0EF02EC182F40401300E82278CEC9C
:1035F0000EF02FC182F40401300E82278CEC0EF005
:1036000030C182F40401300E82278CEC0EF031C1FF
:1036100082F40401300E82278CEC0EF032C182F469
:103620000401300E82278CEC0EF033C182F40401C9
:10363000300E82278CEC0EF0079421EF1DF00784EA
:1036400004014C0E826F8CEC0EF00401320E826F7E
:103650008CEC0EF0C4EC32F0079421EF1DF00784DF
:1036600004014C0E826F8CEC0EF00401330E826F5D
:103670008CEC0EF021EC33F00794BCEF1AF00784C9
:1036800004014C0E826F8CEC0EF00401340E826F3C
:103690008CEC0EF004012C0E826F8CEC0EF02CECF6
:1036A0002EF084C32AF185C32BF186C32CF187C386
:1036B0002DF188C32EF189C32FF18AC330F18BC35A
:1036C00031F18CC332F18DC333F10101296B39EC37
:1036D0002EF0B0EC2DF0100E046F000E056F000EF2
:1036E000066F000E076F01EC2DF000C121F501C13E
:1036F00022F502C123F503C124F51FEC34F038C5CF
:10370000AFF539C5B0F53AC5B1F53BC5B2F53CC525
:10371000B3F53DC5B4F53EC5B5F524EC16F004018E
:103720002C0E826F8CEC0EF03FC500F140C501F10C
:1037300041C502F142C503F10101000E046F000E04
:10374000056F010E066F000E076F21EC2DF08EEC59
:103750002DF02967AEEF1BF0B3EF1BF004012D0E27
:10376000826F8CEC0EF030C182F40401300E82279F
:103770008CEC0EF031C182F40401300E82278CEC07
:103780000EF004012E0E826F8CEC0EF032C182F42A
:103790000401300E82278CEC0EF033C182F4040158
:1037A000300E82278CEC0EF004012C0E826F8CEC14
:1037B0000EF0EBEC2DF043C500F144C501F139ECFE
:1037C00028F004012C0E826F8CEC0EF0EBEC2DF047
:1037D00045C500F18EEC2DF031C182F40401300EAC
:1037E00082278CEC0EF032C182F40401300E822765
:1037F0008CEC0EF033C182F40401300E82278CEC85
:103800000EF004012C0E826F8CEC0EF037C5E8FF31
:10381000E8B806D00401300E826F8CEC0EF005D0B3
:103820000401310E826F8CEC0EF0079421EF1DF035
:103830002CEC2EF085C32AF186C32BF187C32CF123
:1038400088C32DF189C32EF18AC32FF18BC330F1C8
:103850008CC331F18DC332F18EC333F10101296B79
:1038600039EC2EF0B0EC2DF00101010E046F000ECA
:10387000056F000E066F000E076FF0EC2CF0100EB7
:10388000046F000E056F000E066F000E076F01EC4F
:103890002DF000C129F501C12AF502C12BF503C1A4
:1038A0002CF54BEC32F004014C0E826F8CEC0EF0D8
:1038B0000401460E826F8CEC0EF004012C0E826F18
:1038C0008CEC0EF025C500F126C501F127C502F1EB
:1038D00028C503F10101100E046F000E056F000EE4
:1038E000066F000E076F21EC2DF08EEC2DF02AC133
:1038F00082F40401300E82278CEC0EF02BC182F48E
:103900000401300E82278CEC0EF02CC182F40401ED
:10391000300E82278CEC0EF02DC182F40401300EA3
:1039200082278CEC0EF02EC182F40401300E822727
:103930008CEC0EF02FC182F40401300E82278CEC47
:103940000EF030C182F40401300E82278CEC0EF0B0
:1039500031C182F40401300E82278CEC0EF032C1AA
:1039600082F40401300E82278CEC0EF033C182F415
:103970000401300E82278CEC0EF021EF1DF00F9821
:1039800021EC33F035800FEF27F004014C0E826FED
:103990008CEC0EF00401350E826F8CEC0EF00401FD
:1039A0002C0E826F8CEC0EF0EBEC2DF00784B9C579
:1039B00000F107948EEC2DF031C182F40401300E39
:1039C00082278CEC0EF032C182F40401300E822783
:1039D0008CEC0EF033C182F40401300E82278CECA3
:1039E0000EF021EF1DF0E4EC32F0EBEC2DF037C5DA
:1039F00000F18EEC2DF004014C0E826F8CEC0EF079
:103A00000401360E826F8CEC0EF004012C0E826FD6
:103A10008CEC0EF031C182F40401300E82278CEC64
:103A20000EF032C182F40401300E82278CEC0EF0CD
:103A300033C182F40401300E82278CEC0EF021EFAA
:103A40001DF096EC0EF00FEF27F004014C0E826F84
:103A50008CEC0EF00401500E826F8CEC0EF0040121
:103A60002C0E826F8CEC0EF085C32AF186C32BF1ED
:103A700087C32CF188C32DF189C32EF18AC32FF19E
:103A80008BC330F18CC331F18DC332F18EC333F16E
:103A9000010139EC2EF0B0EC2DF003018451530AF2
:103AA0000DE0030184514D0A38E00401780E826F65
:103AB0008CEC0EF096EC0EF00FEF27F00401530E95
:103AC000826F8CEC0EF0250E0C6E00C10BF019EC21
:103AD0000BF0260E0C6E01C10BF019EC0BF0270E4B
:103AE0000C6E02C10BF019EC0BF0280E0C6E03C12A
:103AF0000BF019EC0BF000C157F501C158F502C1EC
:103B000059F503C15AF500C15BF501C15CF502C16D
:103B10005DF503C15EF502EF1EF004014D0E826FEC
:103B20008CEC0EF0290E0C6E00C10BF019EC0BF0B2
:103B300000C15FF500C160F502EF1EF004014C0EFC
:103B4000826F8CEC0EF00401540E826F8CEC0EF040
:103B500004012C0E826F8CEC0EF084C32AF185C315
:103B60002BF186C32CF187C32DF188C32EF189C3B5
:103B70002FF18AC330F18BC331F18DC332F18EC383
:103B800033F1010139EC2EF0B0EC2DF00101000E03
:103B9000046F000E056F010E066F000E076F01EC3B
:103BA0002DF0210E0C6E00C10BF019EC0BF0220E63
:103BB0000C6E01C10BF019EC0BF0230E0C6E02C160
:103BC0000BF019EC0BF0240E0C6E03C10BF019EC8A
:103BD0000BF000C161F501C162F502C163F503C1DB
:103BE00064F502EF1EF004014C0E826F8CEC0EF0B7
:103BF0000401490E826F8CEC0EF004012C0E826FD2
:103C00008CEC0EF0250E30EC0BF0E8CF00F1260E18
:103C100030EC0BF0E8CF01F1270E30EC0BF0E8CFE1
:103C200002F1280E30EC0BF0E8CF03F18EEC2DF012
:103C300051EC2BF00401730E826F8CEC0EF004013A
:103C40002C0E826F8CEC0EF0EBEC2DF0290E30EC8C
:103C50000BF0E8CF00F18EEC2DF051EC2BF00401CD
:103C60006D0E826F8CEC0EF004012C0E826F8CECCA
:103C70000EF05BC500F15CC501F15DC502F15EC5EA
:103C800003F18EEC2DF051EC2BF00401730E826FDA
:103C90008CEC0EF004012C0E826F8CEC0EF0EBEC31
:103CA0002DF060C500F18EEC2DF051EC2BF00401ED
:103CB0006D0E826F8CEC0EF004012C0E826F8CEC7A
:103CC0000EF061C500F162C501F163C502F164C582
:103CD00003F12AEC27F004012C0E826F8CEC0EF01D
:103CE00096EC0EF00FEF27F083C32AF184C32BF17B
:103CF00085C32CF186C32DF187C32EF188C32FF124
:103D000089C330F18AC331F18BC332F18CC333F1F3
:103D1000010139EC2EF0B0EC2DF0160E0C6E00C146
:103D20000BF019EC0BF0170E0C6E01C10BF019EC37
:103D30000BF0180E0C6E02C10BF019EC0BF0190E03
:103D40000C6E03C10BF019EC0BF000C18EF101C138
:103D50008FF102C190F103C191F100C192F101C153
:103D600093F102C194F103C195F156EF1FF083C3A3
:103D70002AF184C32BF185C32CF186C32DF187C3AF
:103D80002EF188C32FF189C330F18AC331F18BC37F
:103D900032F18CC333F1010139EC2EF0B0EC2DF08F
:103DA00000C18EF101C18FF102C190F103C191F107
:103DB00000C192F101C193F102C194F103C195F1E7
:103DC00056EF1FF083C32AF184C32BF185C32CF176
:103DD00086C32DF187C32EF188C32FF189C330F13B
:103DE0008AC331F18CC332F18DC333F1010139EC57
:103DF0002EF0B0EC2DF00101000E046F000E056FE7
:103E0000010E066F000E076F01EC2DF01A0E0C6EFE
:103E100000C10BF019EC0BF01B0E0C6E01C10BF086
:103E200019EC0BF01C0E0C6E02C10BF019EC0BF030
:103E30001D0E0C6E03C10BF019EC0BF000C196F1D6
:103E400001C197F102C198F103C199F156EF1FF03A
:103E500083C32AF184C32BF185C32CF186C32DF1D2
:103E600087C32EF188C32FF189C330F18AC331F1A2
:103E70008CC332F18DC333F1010139EC2EF0B0EC7B
:103E80002DF00101000E046F000E056F010E066F8C
:103E9000000E076F01EC2DF000C196F101C197F102
:103EA00002C198F103C199F156EF1FF0160E30ECE4
:103EB0000BF0E8CF00F1170E30EC0BF0E8CF01F17A
:103EC000180E30EC0BF0E8CF02F1190E30EC0BF0CD
:103ED000E8CF03F18EEC2DF051EC2BF00401730EC2
:103EE000826F8CEC0EF004012C0E826F8CEC0EF0C5
:103EF0008EC100F18FC101F190C102F191C103F1B6
:103F00008EEC2DF051EC2BF00401730E826F8CECD3
:103F10000EF004012C0E826F8CEC0EF01A0E30ECB9
:103F20000BF0E8CF00F11B0E30EC0BF0E8CF01F105
:103F30001C0E30EC0BF0E8CF02F11D0E30EC0BF054
:103F4000E8CF03F12AEC27F004012C0E826F8CECF1
:103F50000EF096C100F197C101F198C102F199C12B
:103F600003F12AEC27F096EC0EF00FEF27F0040196
:103F7000690E826F8CEC0EF004012C0E826F8CECBB
:103F80000EF00101040E006F000E016F000E026FB3
:103F9000000E036F8EEC2DF02CC182F40401300E64
:103FA00082278CEC0EF02DC182F40401300E8227A2
:103FB0008CEC0EF02EC182F40401300E82278CECC2
:103FC0000EF02FC182F40401300E82278CEC0EF02B
:103FD00030C182F40401300E82278CEC0EF031C126
:103FE00082F40401300E82278CEC0EF032C182F490
:103FF0000401300E82278CEC0EF033C182F40401F0
:10400000300E82278CEC0EF004012C0E826F8CECAB
:104010000EF00101060E006F000E016F000E026F20
:10402000000E036F8EEC2DF02CC182F40401300ED3
:1040300082278CEC0EF02DC182F40401300E822711
:104040008CEC0EF02EC182F40401300E82278CEC31
:104050000EF02FC182F40401300E82278CEC0EF09A
:1040600030C182F40401300E82278CEC0EF031C195
:1040700082F40401300E82278CEC0EF032C182F4FF
:104080000401300E82278CEC0EF033C182F404015F
:10409000300E82278CEC0EF004012C0E826F8CEC1B
:1040A0000EF001013D0E006F000E016F000E026F59
:1040B000000E036F8EEC2DF02CC182F40401300E43
:1040C00082278CEC0EF02DC182F40401300E822781
:1040D0008CEC0EF02EC182F40401300E82278CECA1
:1040E0000EF02FC182F40401300E82278CEC0EF00A
:1040F00030C182F40401300E82278CEC0EF031C105
:1041000082F40401300E82278CEC0EF032C182F46E
:104110000401300E82278CEC0EF033C182F40401CE
:10412000300E82278CEC0EF004012C0E826F8CEC8A
:104130000EF0200EF86EF76AF66A04010900F5CF5A
:1041400082F48CEC0EF00900F5CF82F48CEC0EF0CA
:104150000900F5CF82F48CEC0EF00900F5CF82F463
:104160008CEC0EF00900F5CF82F48CEC0EF0090017
:10417000F5CF82F48CEC0EF00900F5CF82F48CECD4
:104180000EF00900F5CF82F48CEC0EF096EC0EF0F8
:104190000FEF27F08351630AD8A40DEF27F0845165
:1041A000610AD8A40DEF27F085516C0AD8A40DEF51
:1041B00027F08651410A3FE08651440A1BE08651B0
:1041C000420AD8B42EEF21F08651350AD8B499EFBF
:1041D00028F08651360AD8B4EEEF28F08651370A17
:1041E000D8B457EF29F08651380AD8B4B5EF29F082
:1041F0000DEF27F00798079A04017A0E826F8CEC76
:104200000EF00401780E826F8CEC0EF00401640E47
:10421000826F8CEC0EF00401550E826F8CEC0EF068
:1042200017EF21F004014C0E826F8CEC0EF096EC2F
:104230000EF00FEF27F00788079A04017A0E826FBD
:104240008CEC0EF00401410E826F8CEC0EF0040138
:10425000610E826F8CEC0EF00BEF21F00798078A4D
:1042600004017A0E826F8CEC0EF00401420E826F14
:104270008CEC0EF00401610E826F8CEC0EF00BEFF3
:1042800021F0010166674CEF21F067674CEF21F0E8
:1042900068674CEF21F0696715D04F6757EF21F041
:1042A000506757EF21F0516757EF21F052670AD05E
:1042B0000101000E006F000E016F000E026F000E74
:1042C000036F120011B80AD00101620E046F010ED3
:1042D000056F000E066F000E076F09D00101A70ED3
:1042E000046F020E056F000E066F000E076F66C1A9
:1042F00000F167C101F168C102F169C103F1F0EC9D
:104300002CF003BFF4EF21F0119A119C0101000E73
:10431000046FA80E056F550E066F020E076F66C17B
:1043200000F167C101F168C102F169C103F166C121
:104330008AF167C18BF168C18CF169C18DF1F0EC34
:104340002CF003BF0BD00101000E8A6FA80E8B6FFB
:10435000550E8C6F020E8D6F118A119C0E0E30EC73
:104360000BF0E8CF18F10F0E30EC0BF0E8CF19F19D
:10437000100E30EC0BF0E8CF1AF1110E30EC0BF010
:10438000E8CF1BF139EC2CF08AC104F18BC105F1A7
:104390008CC106F18DC107F1F0EC2CF00782FDEC29
:1043A0002BF039EC2CF00792FDEC2BF08AC100F1D8
:1043B0008BC101F18CC102F18DC103F10792FDECBB
:1043C0002BF0CC0E046FE00E056F870E066F050E06
:1043D000076FF0EC2CF000C118F101C119F102C116
:1043E0001AF103C11BF140D013AAF9EF21F0138E8B
:1043F000139A119C119A0101800E006F1A0E016F21
:10440000060E026F000E036F4FC104F150C105F19B
:1044100051C106F152C107F1F0EC2CF003AF05D009
:10442000EBEC2DF0118C119A12000E0E30EC0BF00B
:10443000E8CF18F10F0E30EC0BF0E8CF19F1100EA9
:1044400030EC0BF0E8CF1AF1110E30EC0BF0E8CFA6
:104450001BF14FC100F150C101F151C102F152C134
:1044600003F10782FDEC2BF018C100F119C101F135
:104470001AC102F11BC103F112000401730E826F15
:104480008CEC0EF004012C0E826F8CEC0EF0078485
:1044900062C166F163C167F164C168F165C169F128
:1044A0004BC14FF14CC150F14DC151F14EC152F1D0
:1044B00057C159F158C15AF1079463EC22F096ECB8
:1044C0000EF00FEF27F066C100F167C101F168C17E
:1044D00002F169C103F101018EEC2DF051EC2BF0DA
:1044E0000401630E826F8CEC0EF004012C0E826FBF
:1044F0008CEC0EF04FC100F150C101F151C102F13D
:1045000052C103F101018EEC2DF051EC2BF00401AE
:10451000660E826F8CEC0EF004012C0E826F8CEC18
:104520000EF0EBEC2DF059C100F15AC101F101017F
:104530008EEC2DF051EC2BF00401740E826F8CEC9C
:104540000EF0120010820401530E826F8CEC0EF0FC
:1045500004012C0E826F8CEC0EF083C32AF184C30D
:104560002BF185C32CF186C32DF187C32EF188C3AF
:104570002FF189C330F18AC331F18BC332F18CC37F
:1045800033F1010139EC2EF0B0EC2DF000C166F1F1
:1045900001C167F102C168F103C169F18EC32AF15B
:1045A0008FC32BF190C32CF191C32DF192C32EF147
:1045B00093C32FF194C330F195C331F196C332F117
:1045C00097C333F1010139EC2EF0B0EC2DF000C1AE
:1045D0004FF101C150F102C151F103C152F12CEC74
:1045E0002EF099C32FF19AC330F19BC331F19CC3D4
:1045F00032F19DC333F1010139EC2EF0B0EC2DF016
:1046000000C159F101C15AF163EC22F004012C0EF2
:10461000826F8CEC0EF01DEF23F0118E1AA002D0E9
:104620001AAE108C19BE02D019A4108E030182514B
:10463000520A02E10F8201D00F928251750A02E103
:10464000108401D010948251550A02E1108601D0E5
:1046500010968351310A03E11382138402D013921E
:10466000139411A003D011A401D01084078410B2B8
:104670009BEF23F010A47FEF23F0BAC166F1BBC11A
:1046800067F1BCC168F1BDC169F1BEC16AF1BFC1CA
:104690006BF1C0C16CF1C1C16DF1C2C16EF1C3C19A
:1046A0006FF1C4C170F1C5C171F1C6C172F1C7C16A
:1046B00073F1C8C174F1C9C175F1CAC176F1CBC13A
:1046C00077F1CCC178F1CDC179F1CEC17AF1CFC10A
:1046D0007BF1D0C17CF1D1C17DF1D2C17EF1D3C1DA
:1046E0007FF1D4C180F1D5C181F1D6C182F1D7C1AA
:1046F00083F1D8C184F1D9C185F187EF23F062C17C
:1047000066F163C167F164C168F165C169F1BAC15D
:1047100086F1BBC187F1BCC188F1BDC189F14BC134
:104720004FF14CC150F14DC151F14EC152F157C141
:1047300059F158C15AF107940FA0BDEF23F00101C0
:104740009667AAEF23F09767AAEF23F09867AAEF7E
:1047500023F09967AEEF23F0BDEF23F041EC21F099
:1047600096C104F197C105F198C106F199C107F10D
:10477000F0EC2CF003BFD3EF26F041EC21F0010167
:10478000000E046F000E056F010E066F000E076F1E
:1047900021EC2DF011A02AD011A228D08EEC2DF002
:1047A000296701D005D004012D0E826F8CEC0EF02C
:1047B00030C182F40401300E82278CEC0EF031C13E
:1047C00082F40401300E82278CEC0EF032C182F4A8
:1047D0000401300E82278CEC0EF033C182F4040108
:1047E000300E82278CEC0EF096EC0EF012A8C5D09D
:1047F00012981BC01CF01C3A1C42070E1C1600012C
:104800001C50000AD8B489EF24F000011C50010AA2
:10481000D8B415EF24F000011C50020AD8B413EFED
:1048200024F0BBEF24F0BBEF24F0EBEC2DF02BC019
:1048300001F12CC000F1D89001330033D89001333E
:1048400000330101630E046F000E056F000E066F4A
:10485000000E076F21EC2DF0280E046F000E056F7F
:10486000000E066F000E076FF0EC2CF000C12EF06A
:10487000EBEC2DF029C001F1019F019D2AC000F150
:104880000101A40E046F000E056F000E066F000EEE
:10489000076F21EC2DF000C12DF000C104F101C122
:1048A00005F102C106F103C107F1640E006F000EAD
:1048B000016F000E026F000E036FF0EC2CF0050E7E
:1048C000046F000E056F000E066F000E076F21ECDF
:1048D0002DF000C104F101C105F102C106F103C1CF
:1048E00007F1EBEC2DF02EC000F1F0EC2CF000C144
:1048F0002FF02FC0E8FF050F2E5C03E78A84BBEF83
:1049000024F02FC0E8FF0A0F2E5C01E68A94BBEF6B
:1049100024F000C124F101C125F102C126F103C137
:1049200027F1EBEC2DF0F1EC2DF01B501F0BE8CF35
:1049300000F10101640E046F000E056F000E066F9A
:10494000000E076F01EC2DF024C104F125C105F123
:1049500026C106F127C107F1F0EC2CF003BF02D00D
:104960008A9401D08A8424C100F125C101F126C1B5
:1049700002F127C103F10FEF27F000C124F101C1BB
:1049800025F102C126F103C127F110AE4DD0109ED2
:1049900000C108F101C109F102C10AF103C10BF123
:1049A0008EEC2DF030C1DAF131C1DBF132C1DCF136
:1049B00033C1DDF108C100F109C101F10AC102F101
:1049C0000BC103F101016C0E046F070E056F000EA1
:1049D000066F000E076FF0EC2CF003BF04D001014E
:1049E000550EDE6F1CD008C100F109C101F10AC1EA
:1049F00002F10BC103F10101A40E046F060E056F55
:104A0000000E066F000E076FF0EC2CF003BF04D011
:104A100001017F0EDE6F03D00101FF0EDE6F1D8EE0
:104A200011AED3EF26F0119E24C100F125C101F192
:104A300026C102F127C103F111A005D011A203D0B4
:104A40000FB0D3EF26F010A42DEF25F00401750E62
:104A5000826F8CEC0EF032EF25F00401720E826F43
:104A60008CEC0EF004012C0E826F8CEC0EF08EECB0
:104A70002DF0296741EF25F00401200E826F44EFED
:104A800025F004012D0E826F8CEC0EF030C182F403
:104A90000401300E82278CEC0EF031C182F4040147
:104AA000300E82278CEC0EF004012E0E826F8CECFF
:104AB0000EF032C182F40401300E82278CEC0EF02D
:104AC00033C182F40401300E82278CEC0EF0040115
:104AD0006D0E826F8CEC0EF004012C0E826F8CEC4C
:104AE0000EF04FC100F150C101F151C102F152C1AC
:104AF00003F101018EEC2DF051EC2BF00401480E76
:104B0000826F8CEC0EF004017A0E826F8CEC0EF04A
:104B100004012C0E826F8CEC0EF066C100F167C1AF
:104B200001F168C102F169C103F101018EEC2DF0C0
:104B300051EC2BF00401630E826F8CEC0EF004013B
:104B40002C0E826F8CEC0EF066C100F167C101F192
:104B500068C102F169C103F101010A0E046F000E80
:104B6000056F000E066F000E076F01EC2DF0000EB2
:104B7000046F120E056F000E066F000E076F21EC1A
:104B80002DF08EEC2DF02AC182F40401300E822724
:104B90008CEC0EF02BC182F40401300E82278CECD9
:104BA0000EF02CC182F40401300E82278CEC0EF042
:104BB0002DC182F40401300E82278CEC0EF02EC140
:104BC00082F40401300E82278CEC0EF02FC182F4A7
:104BD0000401300E82278CEC0EF030C182F4040107
:104BE000300E82278CEC0EF004012E0E826F8CECBE
:104BF0000EF031C182F40401300E82278CEC0EF0ED
:104C000032C182F40401300E82278CEC0EF033C1E5
:104C100082F40401300E82278CEC0EF00401730E36
:104C2000826F8CEC0EF004012C0E826F8CEC0EF077
:104C3000EBEC2DF059C100F15AC101F139EC28F02B
:104C400013A272EF26F004012C0E826F8CEC0EF092
:104C500086C166F187C167F188C168F189C169F1D0
:104C600041EC21F00101000E046F000E056F010EF2
:104C7000066F000E076F21EC2DF08EEC2DF02967EA
:104C800047EF26F00401200E826F4AEF26F0040160
:104C90002D0E826F8CEC0EF030C182F40401300EC8
:104CA00082278CEC0EF031C182F40401300E822791
:104CB0008CEC0EF004012E0E826F8CEC0EF032C1E3
:104CC00082F40401300E82278CEC0EF033C182F4A2
:104CD0000401300E82278CEC0EF004016D0E826F01
:104CE0008CEC0EF013A499EF26F004012C0E826FC9
:104CF0008CEC0EF013AC87EF26F00401500E826F9F
:104D00008CEC0EF0139C1398139A99EF26F013AEC7
:104D100094EF26F00401460E826F8CEC0EF0139E89
:104D20001398139A99EF26F00401530E826F8CECBE
:104D30000EF00FB29FEF26F00FA0D1EF26F0040186
:104D40002C0E826F8CEC0EF0200EF86EF76AF66A6D
:104D500004010900F5CF82F48CEC0EF00900F5CFC8
:104D600082F48CEC0EF00900F5CF82F48CEC0EF09E
:104D70000900F5CF82F48CEC0EF00900F5CF82F437
:104D80008CEC0EF00900F5CF82F48CEC0EF00900EB
:104D9000F5CF82F48CEC0EF00900F5CF82F48CECA8
:104DA0000EF096EC0EF00F90109E12980FEF27F079
:104DB0000401630E826F8CEC0EF004012C0E826FE6
:104DC0008CEC0EF015EC27F004012C0E826F8CECAD
:104DD0000EF088EC27F004012C0E826F8CEC0EF0A4
:104DE00004EC28F004012C0E826F8CEC0EF0010113
:104DF000F80E006FCD0E016F660E026F030E036F8B
:104E00002AEC27F004012C0E826F8CEC0EF01AECC9
:104E100028F096EC0EF00FEF27F096EC0EF0030161
:104E2000C26B079010921EEF2AF0D8900E0E30EC55
:104E30000BF0E8CF00F10F0E30EC0BF0E8CF01F1F2
:104E4000100E30EC0BF0E8CF02F1110E30EC0BF04D
:104E5000E8CF03F10101000E046F000E056F010E93
:104E6000066F000E076F21EC2DF08EEC2DF02AC19D
:104E700082F40401300E82278CEC0EF02BC182F4F8
:104E80000401300E82278CEC0EF02CC182F4040158
:104E9000300E82278CEC0EF02DC182F40401300E0E
:104EA00082278CEC0EF02EC182F40401300E822792
:104EB0008CEC0EF02FC182F40401300E82278CECB2
:104EC0000EF030C182F40401300E82278CEC0EF01B
:104ED00031C182F40401300E82278CEC0EF0040103
:104EE0002E0E826F8CEC0EF032C182F40401300E73
:104EF00082278CEC0EF033C182F40401300E82273D
:104F00008CEC0EF004016D0E826F8CEC0EF0120032
:104F1000120E30EC0BF0E8CF00F1130E30EC0BF07A
:104F2000E8CF01F1140E30EC0BF0E8CF02F1150ED2
:104F300030EC0BF0E8CF03F101010A0E046F000E14
:104F4000056F000E066F000E076F01EC2DF0000ECE
:104F5000046F120E056F000E066F000E076F21EC36
:104F60002DF08EEC2DF02AC182F40401300E822740
:104F70008CEC0EF02BC182F40401300E82278CECF5
:104F80000EF02CC182F40401300E82278CEC0EF05E
:104F90002DC182F40401300E82278CEC0EF02EC15C
:104FA00082F40401300E82278CEC0EF02FC182F4C3
:104FB0000401300E82278CEC0EF030C182F4040123
:104FC000300E82278CEC0EF004012E0E826F8CECDA
:104FD0000EF031C182F40401300E82278CEC0EF009
:104FE00032C182F40401300E82278CEC0EF033C102
:104FF00082F40401300E82278CEC0EF00401730E53
:10500000826F8CEC0EF012000A0E30EC0BF0E8CF41
:1050100000F10B0E30EC0BF0E8CF01F10C0E30EC90
:105020000BF0E8CF02F10D0E30EC0BF0E8CF03F1FE
:1050300039EF28F0060E30EC0BF0E8CF00F1070E48
:1050400030EC0BF0E8CF01F1080E30EC0BF0E8CFBC
:1050500002F1090E30EC0BF0E8CF03F139EF28F044
:105060000101EBEC2DF0078457C100F158C101F1AB
:1050700007940101E80E046F800E056F000E066FA5
:10508000000E076F01EC2DF0000E046F040E056F8B
:10509000000E066F000E076F21EC2DF0880E046FD6
:1050A000130E056F000E066F000E076FF0EC2CF06C
:1050B0000A0E046F000E056F000E066F000E076FDC
:1050C00021EC2DF08EEC2DF0010129676DEF28F019
:1050D0000401200E826F70EF28F004012D0E826F04
:1050E0008CEC0EF030C182F40401300E82278CEC7F
:1050F0000EF031C182F40401300E82278CEC0EF0E8
:1051000032C182F40401300E82278CEC0EF00401CF
:105110002E0E826F8CEC0EF033C182F40401300E3F
:1051200082278CEC0EF00401430E826F8CEC0EF0A3
:10513000120087C32AF188C32BF189C32CF18AC3DB
:105140002DF18BC32EF18CC32FF18DC330F18EC3A3
:1051500031F190C332F191C333F10101296B39EC84
:105160002EF0B0EC2DF00101000E046F000E056F63
:10517000010E066F000E076F01EC2DF00E0E0C6E87
:1051800000C10BF019EC0BF00F0E0C6E01C10BF00F
:1051900019EC0BF0100E0C6E02C10BF019EC0BF0B9
:1051A000110E0C6E03C10BF019EC0BF004017A0E1A
:1051B000826F8CEC0EF004012C0E826F8CEC0EF0E2
:1051C0000401350E826F8CEC0EF004012C0E826F00
:1051D0008CEC0EF015EC27F017EF21F087C32AF1C5
:1051E00088C32BF189C32CF18AC32DF18BC32EF117
:1051F0008CC32FF18DC330F18EC331F190C332F1E6
:1052000091C333F10101296B39EC2EF0B0EC2DF094
:10521000880E046F130E056F000E066F000E076FE9
:10522000F5EC2CF0000E046F040E056F000E066FF7
:10523000000E076F01EC2DF00101E80E046F800EE7
:10524000056F000E066F000E076F21EC2DF00A0EA1
:105250000C6E00C10BF019EC0BF00B0E0C6E01C1C3
:105260000BF019EC0BF00C0E0C6E02C10BF019ECEC
:105270000BF00D0E0C6E03C10BF019EC0BF00401DA
:105280007A0E826F8CEC0EF004012C0E826F8CEC87
:105290000EF00401360E826F8CEC0EF004012C0E21
:1052A000826F8CEC0EF004EC28F017EF21F087C32E
:1052B0002AF188C32BF189C32CF18AC32DF18BC34A
:1052C0002EF18CC32FF18DC330F18FC331F190C318
:1052D00032F191C333F1010139EC2EF0B0EC2DF035
:1052E000000E046F120E056F000E066F000E076FA2
:1052F00001EC2DF001010A0E046F000E056F000E87
:10530000066F000E076F21EC2DF0120E0C6E00C11F
:105310000BF019EC0BF0130E0C6E01C10BF019EC35
:105320000BF0140E0C6E02C10BF019EC0BF0150E05
:105330000C6E03C10BF019EC0BF004017A0E826FB6
:105340008CEC0EF004012C0E826F8CEC0EF004013C
:10535000370E826F8CEC0EF004012C0E826F8CECF9
:105360000EF088EC27F017EF21F087C32AF188C3ED
:105370002BF189C32CF18AC32DF18BC32EF18CC381
:105380002FF18DC330F18EC331F190C332F191C34F
:1053900033F10101296B39EC2EF0B0EC2DF0880EC1
:1053A000046F130E056F000E066F000E076FF5EC0D
:1053B0002CF0000E046F040E056F000E066F000E39
:1053C000076F01EC2DF00101E80E046F800E056FF0
:1053D000000E066F000E076F21EC2DF0060E0C6E0E
:1053E00000C10BF019EC0BF0070E0C6E01C10BF0B5
:1053F00019EC0BF0080E0C6E02C10BF019EC0BF05F
:10540000090E0C6E03C10BF019EC0BF004017A0EBF
:10541000826F8CEC0EF004012C0E826F8CEC0EF07F
:105420000401380E826F8CEC0EF004012C0E826F9A
:105430008CEC0EF01AEC28F017EF21F007A891EF92
:105440002AF00101800E006F1A0E016F060E026F26
:10545000000E036F4BC104F14CC105F14DC106F1C3
:105460004EC107F1F0EC2CF003BFD7EF2AF04BEC64
:105470002BF04BC100F14CC101F14DC102F14EC105
:1054800003F10782FDEC2BF018C104F119C105F1FD
:105490001AC106F11BC107F1F80E006FCD0E016FA6
:1054A000660E026F030E036FF0EC2CF00E0E0C6E06
:1054B00000C10BF019EC0BF00F0E0C6E01C10BF0DC
:1054C00019EC0BF0100E0C6E02C10BF019EC0BF086
:1054D000110E0C6E03C10BF019EC0BF007840101E7
:1054E000EBEC2DF057C100F158C101F107940A0E01
:1054F0000C6E00C10BF019EC0BF00B0E0C6E01C121
:105500000BF019EC0BF00C0E0C6E02C10BF019EC49
:105510000BF00D0E0C6E03C10BF019EC0BF0D7EF76
:105520002AF007AAD7EF2AF007840101EBEC2DF04F
:1055300057C100F158C101F10794060E0C6E00C16D
:105540000BF019EC0BF0070E0C6E01C10BF019EC0F
:105550000BF0080E0C6E02C10BF019EC0BF0090EEB
:105560000C6E03C10BF019EC0BF0078462C100F163
:1055700063C101F164C102F165C103F10794120E28
:105580000C6E00C10BF019EC0BF0130E0C6E01C188
:105590000BF019EC0BF0140E0C6E02C10BF019ECB1
:1055A0000BF0150E0C6E03C10BF019EC0BF0079805
:1055B000079A0401805181197F0B0DE09EA8FED748
:1055C00014EE00F081517F0BE126E750812B0F0193
:1055D000AD6ED9EF2AF005012F51010A13E081AA1F
:1055E00013EF2BF005012F51000A0AE00FB802EF6C
:1055F0002BF00501306702EF2BF00FB802EF2BF014
:10560000ABEF34F081B813EF2BF01BEC2FF013EF5E
:105610002BF0602F13EF2BF05FC560F50501010E35
:10562000306F3C0E316FCEEF0DF018C100F119C193
:1056300001F11AC102F11BC103F1000E046F000E4B
:10564000056F010E066F000E076F21EC2DF029A1EA
:1056500040EF2BF02051D8B440EF2BF018C100F1EF
:1056600019C101F11AC102F11BC103F1000E046F4F
:10567000000E056F0A0E066F000E076F21EC2DF06D
:1056800012000101045100130551011306510213C8
:105690000751031312000101186B196B1A6B1B6B76
:1056A00012002AC182F40401300E82278CEC0EF025
:1056B0002BC182F40401300E82278CEC0EF02CC139
:1056C00082F40401300E82278CEC0EF02DC182F49E
:1056D0000401300E82278CEC0EF02EC182F40401FE
:1056E000300E82278CEC0EF02FC182F40401300EB4
:1056F00082278CEC0EF030C182F40401300E822738
:105700008CEC0EF031C182F40401300E82278CEC57
:105710000EF032C182F40401300E82278CEC0EF0C0
:1057200033C182F40401300E82278CEC0EF012009B
:105730002FC182F40401300E82278CEC0EF030C1B0
:1057400082F40401300E82278CEC0EF031C182F419
:105750000401300E82278CEC0EF032C182F4040179
:10576000300E82278CEC0EF033C182F40401300E2F
:1057700082278CEC0EF01200060E1F6E060E206EB5
:10578000060E216E1F2EC2EF2BF0202EC2EF2BF043
:10579000212EC2EF2BF08B84020E1F6E020E206EA4
:1057A000020E216E1F2ED2EF2BF0202ED2EF2BF007
:1057B000212ED2EF2BF08B941200FF0E206E20C012
:1057C00021F0030E1F6E8B841F2EE3EF2BF0030ED0
:1057D0001F6E212EE3EF2BF08B9420C021F0030EDF
:1057E0001F6E1F2EF1EF2BF0030E1F6E213EF1EF07
:1057F0002BF0202EDFEF2BF012000101005305E10A
:10580000015303E1025301E1002BC0EC2CF0EBEC5F
:105810002DF03951006F3A51016F420E046F4B0E5B
:10582000056F000E066F000E076F01EC2DF000C132
:1058300004F101C105F102C106F103C107F118C16C
:1058400000F119C101F11AC102F11BC103F107B244
:105850002EEF2CF0F5EC2CF030EF2CF0F0EC2CF0DF
:1058600000C118F101C119F102C11AF103C11BF104
:105870001200EBEC2DF059C100F15AC101F1060EF6
:1058800030EC0BF0E8CF04F1070E30EC0BF0E8CF72
:1058900005F1080E30EC0BF0E8CF06F1090E30EC04
:1058A0000BF0E8CF07F1F0EC2CF000C124F101C1BE
:1058B00025F102C126F103C127F1290E046F000E64
:1058C000056F000E066F000E076F01EC2DF0EE0E57
:1058D000046F430E056F000E066F000E076FF5ECA8
:1058E0002CF024C104F125C105F126C106F127C120
:1058F00007F101EC2DF000C11CF101C11DF102C145
:105900001EF103C11FF1120E30EC0BF0E8CF04F1D1
:10591000130E30EC0BF0E8CF05F1140E30EC0BF069
:10592000E8CF06F1150E30EC0BF0E8CF07F10D0EC5
:10593000006F000E016F000E026F000E036F01EC8E
:105940002DF0180E046F000E056F000E066F000E8E
:10595000076F21EC2DF01CC104F11DC105F11EC122
:1059600006F11FC107F1F5EC2CF06A0E046F2A0E48
:10597000056F000E066F000E076FF0EC2CF01200A2
:10598000BF0EFA6E200E3A6F396BD8900037013790
:1059900002370337D8B0D1EF2CF03A2FC6EF2CF0F6
:1059A00039073A070353D8B412000331070B8009B3
:1059B0003F6F03390F0B010F396F80EC5FF0406FC1
:1059C000390580EC5FF0405D405F396B3F33D8B004
:1059D000392739333FA9E6EF2CF04051392712001F
:1059E000010110EC2EF0D8B012000101035107198B
:1059F000346FD3EC2DF0D8900751031934AF800FDA
:105A000012000101346BF7EC2DF0D8A00DEC2EF054
:105A1000D8B01200E2EC2DF0EBEC2DF01F0E366F3B
:105A200023EC2EF00B35D8B0D3EC2DF0D8A00335F5
:105A3000D8B01200362F10EF2DF034B1FAEC2DF063
:105A400012000101346B0451051106110711000801
:105A5000D8A0F7EC2DF0D8A00DEC2EF0D8B01200A5
:105A6000086B096B0A6B0B6B23EC2EF01F0E366F65
:105A700023EC2EF007510B5DD8A44BEF2DF006510F
:105A80000A5DD8A44BEF2DF00551095DD8A44BEF6A
:105A90002DF00451085DD8A05EEF2DF00451085F91
:105AA0000551D8A0053D095F0651D8A0063D0A5F03
:105AB0000751D8A0073D0B5FD8900081362F38EFF3
:105AC0002DF034B1FAEC2DF0346BF7EC2DF0D890CA
:105AD00027EC2EF007510B5DD8A47BEF2DF006517B
:105AE0000A5DD8A47BEF2DF00551095DD8A47BEFAA
:105AF0002DF00451085DD8A08AEF2DF0003F8AEF09
:105B00002DF0013F8AEF2DF0023F8AEF2DF0032B9D
:105B1000D8B4120034B1FAEC2DF012000101346B4C
:105B2000F7EC2DF0D8B012002CEC2EF0200E366FD2
:105B3000003701370237033711EE33F00A0E376FA3
:105B4000E7360A0EE75CD8B0E76EE552372FA0EFD4
:105B50002DF0362F98EF2DF034B12981D890120016
:105B600001010A0E346F200E366F11EE29F0345108
:105B7000376F0A0ED890E652D8B0E726E732372FB3
:105B8000BBEF2DF00333023301330033362FB5EF73
:105B90002DF0E750FF0FD8A00335D8B0120029B17F
:105BA000FAEC2DF01200045100270551D8B0053D44
:105BB00001270651D8B0063D02270751D8B0073D4E
:105BC000032712000051086F0151096F02510A6F3B
:105BD00003510B6F12000101006B016B026B036B31
:105BE00012000101046B056B066B076B1200033595
:105BF000D8A012000351800B001F011F021F031FBA
:105C0000003F0AEF2EF0013F0AEF2EF0023F0AEFAD
:105C10002EF0032B342B032512000735D8A01200D9
:105C20000751800B041F051F061F071F043F20EFAD
:105C30002EF0053F20EF2EF0063F20EF2EF0072B31
:105C4000342B072512000037013702370337083796
:105C500009370A370B3712000101296B2A6B2B6BAE
:105C60002C6B2D6B2E6B2F6B306B316B326B336B60
:105C7000120001012A510F0B2A6F2B510F0B2B6FB2
:105C80002C510F0B2C6F2D510F0B2D6F2E510F0B15
:105C90002E6F2F510F0B2F6F30510F0B306F315173
:105CA0000F0B316F32510F0B326F33510F0B336FBC
:105CB000120010A806D08994000EC76E220EC66E80
:105CC00005D08984000EC76E220EC66E050EE82E22
:105CD000FED7120010A802D0898401D08994050E45
:105CE000E82EFED7120059EC2EF09E96C69E000EAE
:105CF000C96EFF0E9EB602D0E82EFCD79E96C69EB9
:105D0000000EC96EFF0E9EB602D0E82EFCD7C9CF9A
:105D1000AFF59E96C69E000EC96EFF0E9EB602D0CF
:105D2000E82EFCD7C9CFB0F59E96C69E000EC96E70
:105D3000FF0E9EB602D0E82EFCD7C9CFB1F59E96D5
:105D4000C69E000EC96EFF0E9EB602D0E82EFCD78E
:105D5000C9CFB2F59E96C69E000EC96EFF0E9EB6C6
:105D600002D0E82EFCD7C9CFB3F59E96C69E000E92
:105D7000C96EFF0E9EB602D0E82EFCD7C9CFB4F58F
:105D80009E96C69E000EC96EFF0E9EB602D0E82EED
:105D9000FCD7C9CFB5F56AEC2EF0120059EC2EF005
:105DA0009E96C69E800EC96EFF0E9EB602D0E82E4D
:105DB000FCD79E96C69EAFC5C9FFFF0E9EB602D009
:105DC000E82EFCD79E96C69EB0C5C9FFFF0E9EB6B4
:105DD00002D0E82EFCD79E96C69EB1C5C9FFFF0E25
:105DE0009EB602D0E82EFCD79E96C69EB2C5C9FFCD
:105DF000FF0E9EB602D0E82EFCD79E96C69EB3C577
:105E0000C9FFFF0E9EB602D0E82EFCD79E96C69E16
:105E1000B4C5C9FFFF0E9EB602D0E82EFCD79E96F1
:105E2000C69EB5C5C9FFFF0E9EB602D0E82EFCD7B0
:105E30006AEC2EF0120059EC2EF09E96C69E070ECC
:105E4000C96EFF0E9EB602D0E82EFCD79E96C69E67
:105E5000000EC96EFF0E9EB602D0E82EFCD7C9CF49
:105E6000AFF59E96C69E000EC96EFF0E9EB602D07E
:105E7000E82EFCD7C9CFB0F59E96C69E000EC96E1F
:105E8000FF0E9EB602D0E82EFCD7C9CFB1F59E9684
:105E9000C69E000EC96EFF0E9EB602D0E82EFCD73D
:105EA000C9CFB2F56AEC2EF059EC2EF09E96C69E44
:105EB00023C0C9FFFF0E9EB602D0E82EFCD79E96E7
:105EC000C69E000EC96EFF0E9EB602D0E82EFCD70D
:105ED000C9CFB6F56AEC2EF0120059EC2EF09E9662
:105EE000C69E870EC96EFF0E9EB602D0E82EFCD766
:105EF0009E96C69EAFC5C9FFFF0E9EB602D0E82E85
:105F0000FCD79E96C69EB0C5C9FFFF0E9EB602D0B6
:105F1000E82EFCD79E96C69EB1C5C9FFFF0E9EB661
:105F200002D0E82EFCD79E96C69EB2C5C9FFFF0ED2
:105F30009EB602D0E82EFCD76AEC2EF059EC2EF07B
:105F40009E96C69E24C0C9FFFF0E9EB602D0E82EC4
:105F5000FCD79E96C69EB6C5C9FFFF0E9EB602D060
:105F6000E82EFCD76AEC2EF0120059EC2EF09E962B
:105F7000C69E870EC96EFF0E9EB602D0E82EFCD7D5
:105F80009E96C69E000EC96EFF0E9EB602D0E82EEB
:105F9000FCD79E96C69E800EC96EFF0E9EB602D09E
:105FA000E82EFCD79E96C69E800EC96EFF0E9EB64A
:105FB00002D0E82EFCD79E96C69E800EC96EFF0EBC
:105FC0009EB602D0E82EFCD76AEC2EF0120059ECF7
:105FD0002EF09E96C69E870EC96EFF0E9EB602D00C
:105FE000E82EFCD79E96C69E000EC96EFF0E9EB68A
:105FF00002D0E82EFCD79E96C69E000EC96EFF0EFC
:106000009EB602D0E82EFCD79E96C69E800EC96E24
:10601000FF0E9EB602D0E82EFCD79E96C69E800E3E
:10602000C96EFF0E9EB602D0E82EFCD76AEC2EF0A9
:10603000120010A817D059EC2EF09E96C69E8F0E17
:10604000C96EFF0E9EB602D0E82EFCD79E96C69E65
:10605000000EC96EFF0E9EB602D0E82EFCD76AEC89
:106060002EF012001BEC2FF0120010A82DD059ECCE
:106070002EF09E96C69E24C0C9FFFF0E9EB602D08B
:10608000E82EFCD79E96C69E450EC96EFF0E9EB6A4
:1060900002D0E82EFCD76AEC2EF059EC2EF09E963A
:1060A000C69E8F0EC96EFF0E9EB602D0E82EFCD79C
:1060B0009E96C69E000EC96EFF0E9EB602D0E82EBA
:1060C000FCD76AEC2EF0120059EC2EF09E96C69E7C
:1060D00024C0C9FFFF0E9EB602D0E82EFCD79E96C4
:1060E000C69E010EC96EFF0E9EB602D0E82EFCD7EA
:1060F0006AEC2EF059EC2EF09E96C69E910EC96E5B
:10610000FF0E9EB602D0E82EFCD79E96C69EA50E28
:10611000C96EFF0E9EB602D0E82EFCD76AEC2EF0B8
:10612000120059EC2EF09E96C69E24C0C9FFFF0EA9
:106130009EB602D0E82EFCD79E96C69E810EC96EF2
:10614000FF0E9EB602D0E82EFCD76AEC2EF01200AD
:1061500059EC2EF09E96C69E24C0C9FFFF0E9EB637
:1061600002D0E82EFCD79E96C69E010EC96EFF0E89
:106170009EB602D0E82EFCD76AEC2EF0120059EC45
:106180002EF09E96C69E910EC96EFF0E9EB602D050
:10619000E82EFCD79E96C69EA50EC96EFF0E9EB633
:1061A00002D0E82EFCD76AEC2EF0120059EC2EF04B
:1061B0009E96C69E910EC96EFF0E9EB602D0E82E28
:1061C000FCD79E96C69E000EC96EFF0E9EB602D0EC
:1061D000E82EFCD76AEC2EF012000501256B266B29
:1061E000276B286B899A400EC76E200EC66E9E964E
:1061F000C69E030EC96EFF0E9EB602D0E82EFCD7D7
:106200009E96C69E27C5C9FFFF0E9EB602D0E82EF9
:10621000FCD79E96C69E26C5C9FFFF0E9EB602D02D
:10622000E82EFCD79E96C69E25C5C9FFFF0E9EB6DA
:1062300002D0E82EFCD79E96C69EC952FF0E9EB68F
:1062400002D0E82EFCD7898A0F01C950FF0A01E16C
:10625000120005012E51130A05E005012E51170AFF
:106260000CE012000501F00E256FFF0E266F0F0ED9
:10627000276F000E286F46EF31F00501F00E256FF5
:10628000FF0E266FFF0E276F000E286F899A400EB3
:10629000C76E200EC66E9E96C69E030EC96EFF0E7A
:1062A0009EB602D0E82EFCD79E96C69E27C5C9FF93
:1062B000FF0E9EB602D0E82EFCD79E96C69E26C53F
:1062C000C9FFFF0E9EB602D0E82EFCD79E96C69E52
:1062D00025C5C9FFFF0E9EB602D0E82EFCD79E96BC
:1062E000C69EC952FF0E9EB602D0E82EFCD7898A00
:1062F0000F01C950FF0A1DE005012E51130A05E0E8
:1063000005012E51170A0BE012000501000E256F42
:10631000000E266F100E276F000E286F1200050169
:10632000000E256F000E266F000E276F010E286FDE
:1063300012000501256B266B276B286B05012E517A
:10634000130A05E005012E51170A0CE012000501A1
:10635000000E216F000E226F080E236F000E246FB7
:10636000BBEF31F00501000E216F000E226F800E91
:10637000236F000E246F21C500F122C501F123C552
:1063800002F124C503F125C504F126C505F127C591
:1063900006F128C507F141EC2BF000C125F501C13C
:1063A00026F502C127F503C128F5899A400EC76E6C
:1063B000200EC66E9E96C69E030EC96EFF0E9EB63A
:1063C00002D0E82EFCD79E96C69E27C5C9FFFF0EB9
:1063D0009EB602D0E82EFCD79E96C69E26C5C9FF63
:1063E000FF0E9EB602D0E82EFCD79E96C69E25C50F
:1063F000C9FFFF0E9EB602D0E82EFCD79E96C69E21
:10640000C952FF0E9EB602D0E82EFCD7898AC95029
:10641000FF0A08E104C125F505C126F506C127F5E7
:1064200007C128F5D89005012433233322332133C3
:106430002151F00B216F216725EF32F0226725EF04
:1064400032F0236725EF32F02467BBEF31F005010E
:10645000100E2527E86A2623E86A2723E86A2823FE
:106460001200E86A05012E51130A06E005012E51BB
:10647000170A0BE0020E120005012851000A03E181
:106480002751F00B07E0010E120005012851000A08
:1064900001E0010E120029C500F12AC501F12BC54A
:1064A00002F12CC503F125C504F126C505F127C568
:1064B00006F128C507F1F0EC2CF003BF120031EC17
:1064C00032F0D8A4C3EF32F0899A400EC76E200E86
:1064D000C66E9E96C69E060EC96EFF0E9EB602D072
:1064E000E82EFCD7898A899A9E96C69E020EC96EAE
:1064F000FF0E9EB602D0E82EFCD79E96C69E27C5FC
:10650000C9FFFF0E9EB602D0E82EFCD79E96C69E0F
:1065100026C5C9FFFF0E9EB602D0E82EFCD79E9678
:10652000C69E25C5C9FFFF0E9EB602D0E82EFCD739
:106530009E96C69E000EC96EFF0E9EB602D0E82E35
:10654000FCD7898A899A9E96C69E050EC96EFF0E53
:106550009EB602D0E82EFCD79E96C69EC952FF0E6C
:106560009EB602D0E82EFCD7C9B0ACEF32F0898AD3
:106570000501100E2527E86A2623E86A2723E86A22
:1065800028234BEF32F01200899A400EC76E200E7E
:10659000C66E9E96C69E060EC96EFF0E9EB602D0B1
:1065A000E82EFCD7898A899A9E96C69EC70EC96E28
:1065B000FF0E9EB602D0E82EFCD7898A0501256B16
:1065C000266B276B286B1200899A400EC76E200E2F
:1065D000C66E9E96C69E050EC96EFF0E9EB602D072
:1065E000E82EFCD79E96C69EC952FF0E9EB602D0DC
:1065F000E82EFCD7C9CF37F5898A1200899A400E58
:10660000C76E200EC66E9E96C69EB90EC96EFF0E50
:106610009EB602D0E82EFCD7898A1200899A400ED5
:10662000C76E200EC66E9E96C69EAB0EC96EFF0E3E
:106630009EB602D0E82EFCD7898AFF0EE82EFED740
:10664000120031EC32F0D8A41200899A400EC76EC5
:10665000200EC66E9E96C69E030EC96EFF0E9EB697
:1066600002D0E82EFCD79E96C69E27C5C9FFFF0E16
:106670009EB602D0E82EFCD79E96C69E26C5C9FFC0
:10668000FF0E9EB602D0E82EFCD79E96C69E25C56C
:10669000C9FFFF0E9EB602D0E82EFCD79E96C69E7E
:1066A000C952FF0E9EB602D0E82EFCD7898A0F0190
:1066B000C950FF0AD8A41EEF34F00501FE0E376F53
:1066C00035A0379973EC2EF0AFC538F5B0C539F564
:1066D000B1C53AF5B2C53BF5B3C53CF5B4C53DF51A
:1066E000B5C53EF50784BAC166F1BBC167F1BCC14F
:1066F00068F1BDC169F14BC14FF14CC150F14DC1C1
:1067000051F14EC152F157C159F158C15AF141EC02
:1067100021F000C13FF501C140F502C141F503C1BF
:1067200042F5050161679CEF33F062679CEF33F03F
:1067300063679CEF33F06467A0EF33F0ADEF33F0A5
:1067400061C504F162C505F163C506F164C507F1D1
:10675000F0EC2CF003BF1EEF34F059C143F55AC1E1
:1067600044F5B9C545F5BAC546F507940501110EBE
:10677000326F899A400EC76E200EC66E9E96C69ED8
:10678000060EC96EFF0E9EB602D0E82EFCD7898A8F
:10679000899A9E96C69E020EC96EFF0E9EB602D0C4
:1067A000E82EFCD79E96C69E27C5C9FFFF0E9EB653
:1067B00002D0E82EFCD79E96C69E26C5C9FFFF0EC6
:1067C0009EB602D0E82EFCD79E96C69E25C5C9FF70
:1067D000FF0E9EB602D0E82EFCD725EE37F0322F02
:1067E00002D0FEEF33F09E96C69EDECFC9FFFF0EAD
:1067F0009EB602D0E82EFCD7EFEF33F0898A899A53
:106800009E96C69E050EC96EFF0E9EB602D0E82E5D
:10681000FCD79E96C69EC952FF0E9EB602D0E82EA9
:10682000FCD7C9B009EF34F0898A0501100E25277D
:10683000E86A2623E86A2723E86A2823120021C58C
:1068400000F122C501F123C502F124C503F1899AA3
:10685000400EC76E200EC66E9E96C69E0B0EC96E6B
:10686000FF0E9EB602D0E82EFCD79E96C69E02C1B1
:10687000C9FFFF0E9EB602D0E82EFCD79E96C69E9C
:1068800001C1C9FFFF0E9EB602D0E82EFCD79E962E
:10689000C69E00C1C9FFFF0E9EB602D0E82EFCD7EF
:1068A0009E96C69EC952FF0E9EB602D0E82EFCD719
:1068B00025EE37F00501100E326F9E96C69EC95226
:1068C000FF0E9EB602D0E82EFCD7C9CFDEFF322FD6
:1068D0005DEF34F0898A1200899A400EC76E200E4F
:1068E000C66E9E96C69E900EC96EFF0E9EB602D0D4
:1068F000E82EFCD79E96C69E000EC96EFF0E9EB671
:1069000002D0E82EFCD79E96C69E000EC96EFF0EE2
:106910009EB602D0E82EFCD79E96C69E000EC96E8B
:10692000FF0E9EB602D0E82EFCD79E96C69EC95298
:10693000FF0E9EB602D0E82EFCD7C9CF2DF59E964D
:10694000C69EC952FF0E9EB602D0E82EFCD7C9CF14
:106950002EF5898A1200BCEC2BF0B9C5E8FFD708E8
:1069600002E3BCEC2BF0B9C5E8FFC80802E3BCECBD
:106970002BF0B9C5E8FFB90802E3BCEC2BF0B9C5B0
:10698000E8FFAA0802E3BCEC2BF0B9C5E8FF9B08BE
:1069900002E3BCEC2BF0FEEC32F0F29CF29E8B9406
:1069A000C69AC2909482948C720ED36ED3A4FED7F2
:1069B00089968A909390F29AF2949D909E909D92DF
:1069C0009E92F298F29219EC30F0FF0EE8CF00F0B0
:1069D000E82EFED7002EFCD7F290F286815081A8D7
:1069E000F4EF34F0F29E0300700ED36EF296F29044
:0E69F000010E356E0380DDEC2BF065EF0BF031
:10BF0000E844F926000C160C2B0C3F0C520C640C68
:10BF1000760C860C960CA50CB30CC10CCF0CDC0C6B
:06BF2000E80CF40C000C1B
:0200000400F00A
:0100C800FE39
:00000001FF
